:020000040000FA
:1000000002EF00F00F013F0E926E000E936E000E95
:10001000946E030E956E0F0E966E000E386F000EE6
:10002000396F000E3A6F000E3B6F000E3C6F806A16
:10003000816A826A836A846A896A8A6A8B6A8C6A3C
:100040008D6A00018B8C006A016A026A036A046A85
:10005000056A066A076A086A096A0A6A0B6A0C6A0C
:100060000D6A0E6A0F6A106A116A126A136A146ABC
:10007000156A166A176A186A196A1A6A1B6A1C6A6C
:100080001D6A1E6A1F6A206A216A226A236A256A1B
:10009000266A276A296A246A286A2A6A2B6A2C6ACD
:1000A0002D6A2E6A2F6A306A316A326A336A346A7C
:1000B000356A366A376A386A396A3A6A3C6A3B6A2C
:1000C0003D6A3E6A3F6A406A416A426A436A446ADC
:1000D000456A466A476A486A496A4A6A4B6A4C6A8C
:1000E0004D6A4E6A506A516A526A536A546A556A36
:1000F000566A576A586A596A5A6A6AEC37F06AEC63
:1001000037F06AEC37F06AEC37F02BEC2BF0C00ECE
:100110008A6E8C9C8C9E8C8A8C9A2AEC2CF03F0EDA
:100120008A6E8C9C8C9E8C8A8C9A4DEC2CF08B8ADF
:100130002EEC2BF092EC37F0000EAA6E000EA96E9A
:10014000A69EA69CA68000000000A850116E000E7E
:10015000AA6E010EA96EA69EA69CA68000000000B5
:10016000A850126E000EAA6E020EA96EA69EA69C44
:10017000A68000000000A850136E000EAA6E030EA9
:10018000A96EA69EA69CA68000000000A850146E32
:10019000000EAA6E040EA96EA69EA69CA680000064
:1001A0000000A850156E000EAA6E050EA96EA69E40
:1001B000A69CA68000000000A850166E000EAA6E35
:1001C000060EA96EA69EA69CA68000000000A85060
:1001D000176E000EAA6E070EA96EA69EA69CA6809C
:1001E00000000000A850186E000EAA6E080EA96E3E
:1001F000A69EA69CA68000000000A850196E000EC6
:10020000AA6E090EA96EA69EA69CA68000000000FC
:10021000A8501A6E000EAA6E0A0EA96EA69EA69C83
:10022000A68000000000A8504C6E6AEC2CF0AFECE9
:100230002DF01D504E6E4CA423EF01F083A223EF4E
:1002400001F045EC36F0AFEC2DF080B280B650EF07
:1002500001F0070E5A5CD8B431EF01F05A2A52EF80
:1002600001F05A6A3EB652EF01F01550380B406E5D
:10027000380E405CD8B441EF01F0080E402643EF41
:1002800001F0000E406E1550C70B156E4050151250
:100290004CB262EC36F06AEC2CF03E8652EF01F084
:1002A0003E965A6A80B47CEF01F0070E595CD8B4D0
:1002B0005DEF01F0592A7EEF01F0596A3EB47EEFFE
:1002C00001F01550380B406E000E405CD8B46DEF55
:1002D00001F0080E405E6FEF01F0380E406E1550D1
:1002E000C70B156E405015124CB262EC36F06AEC3A
:1002F0002CF03E847EEF01F03E94596A4CB440EC01
:1003000036F080B29EEF01F0070E585CD8B48CEF47
:1003100001F0582AA0EF01F0586A3EB2A0EF01F0B8
:10032000040E415CD8B498EF01F0412A99EF01F036
:10033000416A4DEC2CF03E82A0EF01F03E92586AEB
:10034000000E415CD8B4BBEF01F0010E415CD8B4A3
:10035000B0EF0BF0020E415CD8B4E6EF11F0030EE3
:10036000415CD8B41EEF21F0040E415CD8B4CAEF52
:1003700026F023EF01F025EC2BF0410E31EC2BF0B1
:10038000B80E4AEC2BF0700E63EC2BF0100E63EC01
:100390002BF0100E63EC2BF0100E63EC2BF0000E24
:1003A00063EC2BF089EC46F0000E63EC2BF0C9EC0B
:1003B00045F0000E63EC2BF0A9EC45F0000E63EC69
:1003C0002BF0C9EC45F0000E63EC2BF009EC46F085
:1003D000000E63EC2BF0C9EC46F0000E63EC2BF042
:1003E000C9EC45F0000E63EC2BF089EC46F0B9EC5B
:1003F00048F099EC46F028EC2BF0400E31EC2BF055
:10040000B80E4AEC2BF0A9EC46F0000E63EC2BF092
:1004100089EC45F0000E63EC2BF0A9EC46F0000EE1
:1004200063EC2BF0B9EC46F0000E63EC2BF099EC8A
:1004300046F0000E63EC2BF0082A210E085CD8B4BD
:1004400027EF02F0100E63EC2BF01CEF02F0086AAD
:10045000700E63EC2BF025EC2BF0400E31EC2BF002
:10046000BA0E4AEC2BF01DA852EF02F0B9EC48F09E
:10047000B9EC48F0B9EC48F0B9EC48F0000E63EC88
:100480002BF0B9EC48F0000E63EC2BF0B9EC48F01F
:10049000000E63EC2BF0B9EC48F0000E63EC2BF08F
:1004A0007CEF02F01BA49EEF02F0FF0E63EC2BF03A
:1004B000E9EC47F0FF0E63EC2BF0F9EC47F0FF0E90
:1004C00063EC2BF0FF0E63EC2BF0FF0E63EC2BF0D4
:1004D00039EC48F0FF0E63EC2BF039EC47F0FF0EDF
:1004E00063EC2BF0D9EC47F0FF0E63EC2BF039EC0A
:1004F00048F0FF0E63EC2BF0082A1A0E085CD8B403
:1005000087EF02F0000E63EC2BF07CEF02F0086A3C
:1005100028EC2BF0400E31EC2BF0BA0E4AEC2BF00D
:10052000082A070E085CD8B49BEF02F0000E63ECBB
:100530002BF090EF02F0086A25EF03F0FF0E63EC5A
:100540002BF039EC48F0FF0E63EC2BF039EC47F060
:10055000FF0E63EC2BF0D9EC47F0FF0E63EC2BF0B1
:1005600039EC48F0FF0E63EC2BF0000E63EC2BF03F
:10057000000E63EC2BF01BA2EEEF02F0FF0E63EC1B
:100580002BF0F9EC47F0FF0E63EC2BF029EC48F070
:10059000FF0E63EC2BF099EC47F0FF0E63EC2BF0B1
:1005A00079EC47F0FF0E63EC2BF0E9EC47F0FF0E1F
:1005B00063EC2BF019EC47F0FF0E63EC2BF028EC0A
:1005C0002BF0400E31EC2BF0BA0E4AEC2BF0C9ECBC
:1005D00047F0FF0E63EC2BF025EF03F0FF0E63EC0A
:1005E0002BF039EC47F0FF0E63EC2BF0F9EC47F001
:1005F000FF0E63EC2BF009EC48F0FF0E63EC2BF0E0
:1006000099EC48F0FF0E63EC2BF0082A0D0E085C05
:10061000D8B410EF03F0000E63EC2BF005EF03F0FD
:10062000086A28EC2BF0400E31EC2BF0BA0E4AECA5
:100630002BF0082A070E085CD8B424EF03F0000E54
:1006400063EC2BF019EF03F0086A28EC2BF0480E4E
:1006500031EC2BF0BA0E4AEC2BF01DB847EF03F04B
:100660001BA647EF03F0FF0E63EC2BF009EC48F0FC
:10067000FF0E63EC2BF029EC48F0FF0E63EC2BF03F
:10068000F9EC47F0FF0E63EC2BF053EF03F0082A70
:10069000140E085CD8B452EF03F0000E63EC2BF09C
:1006A00047EF03F0086A28EC2BF05D0E31EC2BF0DD
:1006B000BA0E4AEC2BF01DB87AEF03F01BB07AEFBC
:1006C00003F0FF0E63EC2BF059EC47F0FF0E63ECE8
:1006D0002BF0D9EC47F0FF0E63EC2BF009EC48F05F
:1006E000FF0E63EC2BF089EC47F0FF0E63EC2BF070
:1006F00086EF03F0082A1A0E085CD8B485EF03F0E1
:10070000000E63EC2BF07AEF03F0086A25EC2BF077
:10071000400E31EC2BF0B90E4AEC2BF01DB805EF72
:1007200005F01CB69FEF03F01CB8CDEF03F01CBA28
:10073000FBEF03F01CBC2BEF04F005EF05F0FF0E00
:1007400063EC2BF049EC47F0FF0E63EC2BF049EC27
:1007500048F0FF0E63EC2BF039EC48F0FF0E63EC31
:100760002BF0FF0E63EC2BF0FF0E39EC47F0FF0E81
:1007700063EC2BF049EC47F0FF0E63EC2BF0082AFA
:10078000110E085CD8B4CAEF03F0000E63EC2BF036
:10079000BFEF03F0086A11EF05F0FF0E63EC2BF0DA
:1007A00049EC47F0FF0E63EC2BF049EC48F0FF0EEC
:1007B00063EC2BF039EC48F0FF0E63EC2BF0FF0EEE
:1007C00063EC2BF0FF0EC9EC47F0FF0E63EC2BF04F
:1007D00049EC47F0FF0E63EC2BF0082A110E085C81
:1007E000D8B4F8EF03F0000E63EC2BF0EDEF03F05C
:1007F000086A11EF05F0FF0E63EC2BF099EC47F05F
:10080000FF0E63EC2BF059EC47F0FF0E63EC2BF07E
:1008100039EC47F0FF0E63EC2BF0A9EC43F0FF0E30
:1008200063EC2BF059EC43F0FF0E63EC2BF0D9ECAA
:1008300043F0FF0E63EC2BF079EC43F0FF0E63EC1A
:100840002BF0B9EC43F0FF0E63EC2BF0000E63ECE1
:100850002BF011EF05F0FF0E63EC2BF009EC48F0E4
:10086000FF0E63EC2BF039EC47F0FF0E63EC2BF03E
:10087000D9EC47F0FF0E63EC2BF0000E63EC2BF08D
:100880002B50526E529E010E525CD8B465EF04F0AC
:10089000490E525CD8B48DEF04F0030E525CD8B40C
:1008A000B5EF04F0430E525CD8B4DDEF04F0082A33
:1008B0001E0E085CD8B462EF04F0000E63EC2BF05F
:1008C00057EF04F0086A11EF05F0000E63EC2BF00F
:1008D000FF0E63EC2BF039EC47F0FF0E63EC2BF0CE
:1008E00049EC47F0FF0E63EC2BF0B9EC48F0000E3A
:1008F00063EC2BF0B9EC48F0000E63EC2BF0000E2B
:1009000063EC2BF0000E63EC2BF0000E63EC2BF08D
:10091000000E63EC2BF011EF05F0000E63EC2BF0F2
:10092000FF0E63EC2BF0D9EC47F0FF0E63EC2BF0DD
:1009300049EC47F0FF0E63EC2BF0B9EC48F0000EE9
:1009400063EC2BF0B9EC48F0000E63EC2BF0000EDA
:1009500063EC2BF0000E63EC2BF0000E63EC2BF03D
:10096000000E63EC2BF011EF05F0000E63EC2BF0A2
:10097000FF0E63EC2BF049EC47F0FF0E63EC2BF01D
:1009800019EC47F0FF0E63EC2BF049EC48F0FF0E3A
:1009900063EC2BF0B9EC48F0000E63EC2BF0000E8A
:1009A00063EC2BF0000E63EC2BF0000E63EC2BF0ED
:1009B000000E63EC2BF011EF05F0000E63EC2BF052
:1009C000FF0E63EC2BF049EC47F0FF0E63EC2BF0CD
:1009D00039EC47F0FF0E63EC2BF039EC47F0FF0EDB
:1009E00063EC2BF0B9EC48F0000E63EC2BF0000E3A
:1009F00063EC2BF0000E63EC2BF0000E63EC2BF09D
:100A0000000E63EC2BF011EF05F0082A320E085CA3
:100A1000D8B410EF05F0000E63EC2BF005EF05F0F5
:100A2000086A25EC2BF0730E31EC2BF0B90E4AEC72
:100A30002BF01DB84FEF05F01CA24FEF05F0FF0E95
:100A400063EC2BF039EC48F0FF0E63EC2BF099ECE3
:100A500047F0FF0E63EC2BF028EC2BF0400E31EC4E
:100A60002BF0B90E4AEC2BF0C9EC47F0FF0E63EC0B
:100A70002BF059EC47F0FF0E63EC2BF0E9EC47F05C
:100A8000FF0E63EC2BF039EC47F0FF0E63EC2BF01C
:100A900059EC47F0FF0E63EC2BF06FEF05F0082ADE
:100AA0000E0E085CD8B45AEF05F0000E63EC2BF084
:100AB0004FEF05F0086A28EC2BF0400E31EC2BF0DC
:100AC000B90E4AEC2BF0082A1F0E085CD8B46EEF62
:100AD00005F0000E63EC2BF063EF05F0086A28ECDC
:100AE0002BF0600E31EC2BF0B90E4AEC2BF01DB858
:100AF0009FEF05F01CA09FEF05F0FF0E63EC2BF0BD
:100B000089EC47F0FF0E63EC2BF099EC47F0FF0EF9
:100B100063EC2BF0FF0E63EC2BF0FF0E63EC2BF07D
:100B200069EC47F0FF0E63EC2BF039EC48F0FF0E58
:100B300063EC2BF0000E63EC2BF0ABEF05F0082A12
:100B40001C0E085CD8B4AAEF05F0000E63EC2BF085
:100B50009FEF05F0086A25EC2BF0400E31EC2BF0EE
:100B6000BB0E4AEC2BF04CB0BBEF05F01D504E6EA7
:100B70004F6AD0EF05F01D504E5CD8A43F9A000E8E
:100B80004F5CD8A4C6EF05F01D504E6E3FBAD0EFB3
:100B900005F0000E4E5CD8B4D0EF05F07FEC3AF0D3
:100BA000000E4E5CD8A4D9EF05F0FDEC3AF023EF2F
:100BB00006F0400E4E5CD8A4E2EF05F01DEC3BF0D1
:100BC00023EF06F0200E4E5CD8A4EBEF05F03EECD0
:100BD0003BF023EF06F0100E4E5CD8A4F4EF05F0C6
:100BE0005FEC3BF023EF06F0080E4E5CD8A4FDEF5F
:100BF00005F097EC3BF023EF06F0020E4E5CD8A414
:100C000006EF06F0E5EC3BF023EF06F0010E4E5C3C
:100C1000D8A40FEF06F033EC3CF023EF06F0FF0E04
:100C200063EC2BF0B3EC3CF04E50B0EC39F0FF0E1F
:100C300063EC2BF0FF0E63EC2BF012EC3AF0B9EC06
:100C400048F0B9EC48F025EC2BF0400E31EC2BF0DD
:100C5000BD0E4AEC2BF0000E63EC2BF0D9EC45F006
:100C6000000E63EC2BF099EC46F0000E63EC2BF0D9
:100C7000280E63EC2BF0280E63EC2BF0280E63ECAF
:100C80002BF0280E63EC2BF0280E63EC2BF0000EFB
:100C900063EC2BF025EC2BF0530E31EC2BF0BD0E5A
:100CA0004AEC2BF05E0E295CD8A476EF06F0000E1D
:100CB00063EC2BF0B9EC48F0000E63EC2BF0B9ECD0
:100CC00048F0000E63EC2BF0000E63EC2BF0000EEE
:100CD00063EC2BF0D9EC42F0000E63EC2BF0C9EC86
:100CE00042F0000E63EC2BF09BEF08F05D0E295CE8
:100CF000D8A49AEF06F0000E63EC2BF0B9EC48F0A4
:100D0000000E63EC2BF0B9EC48F0000E63EC2BF016
:100D1000000E63EC2BF0000E63EC2BF0D9EC42F0EC
:100D2000000E63EC2BF0C9EC42F0000E63EC2BF0EC
:100D30009BEF08F0440E295CD8A4BEEF06F0000E2D
:100D400063EC2BF0B9EC48F0000E63EC2BF0E9EC0F
:100D500042F0000E63EC2BF0E9EC42F0000E63EC85
:100D60002BF0400E63EC2BF0000E63EC2BF0B9EC93
:100D700042F0000E63EC2BF09BEF08F0450E295C6F
:100D8000D8A4E2EF06F0000E63EC2BF0B9EC48F0CB
:100D9000000E63EC2BF0E9EC42F0000E63EC2BF05C
:100DA000E9EC42F0000E63EC2BF0400E63EC2BF00C
:100DB000000E63EC2BF0B9EC42F0000E63EC2BF06C
:100DC0009BEF08F03E0E295CD8A406EF07F0000E5A
:100DD00063EC2BF0B9EC48F0000E63EC2BF0B9ECAF
:100DE00048F0000E63EC2BF0000E63EC2BF0000ECD
:100DF00063EC2BF0E9EC42F0000E63EC2BF029ECF5
:100E000043F0000E63EC2BF09BEF08F03F0E295CE3
:100E1000D8A42AEF07F0000E63EC2BF0B9EC48F0F1
:100E2000000E63EC2BF0B9EC48F0000E63EC2BF0F5
:100E3000000E63EC2BF0000E63EC2BF0E9EC42F0BB
:100E4000000E63EC2BF029EC43F0000E63EC2BF06A
:100E50009BEF08F0220E295CD8A44EEF07F0000E9D
:100E600063EC2BF0B9EC48F0FF0E63EC2BF0C9EC0F
:100E700043F0FF0E63EC2BF0C9EC43F0FF0E63EC84
:100E80002BF0BF0E63EC2BF0FF0E63EC2BF069EC44
:100E900043F0FF0E63EC2BF09BEF08F0230E295C70
:100EA000D8A472EF07F0000E63EC2BF0B9EC48F019
:100EB000FF0E63EC2BF0C9EC43F0FF0E63EC2BF05C
:100EC000C9EC43F0FF0E63EC2BF0BF0E63EC2BF08C
:100ED000FF0E63EC2BF069EC43F0FF0E63EC2BF09C
:100EE0009BEF08F01F0E295CD8A496EF07F0000EC8
:100EF00063EC2BF0B9EC48F0000E63EC2BF0B9EC8E
:100F000048F0000E63EC2BF0000E63EC2BF0FF0EAC
:100F100063EC2BF0D9EC43F0FF0E63EC2BF0A9EC63
:100F200043F0FF0E63EC2BF09BEF08F0200E295CE2
:100F3000D8A4BAEF07F0000E63EC2BF0B9EC48F040
:100F4000000E63EC2BF0B9EC48F0000E63EC2BF0D4
:100F5000000E63EC2BF0FF0E63EC2BF0D9EC43F0AA
:100F6000FF0E63EC2BF0A9EC43F0FF0E63EC2BF0CB
:100F70009BEF08F0110E295CD8A4DEEF07F0FF0EFE
:100F800063EC2BF059EC43F0FF0E63EC2BF0B9EC63
:100F900043F0FF0E63EC2BF0A9EC43F0FF0E63EC83
:100FA0002BF0BF0E63EC2BF0FF0E63EC2BF089EC03
:100FB00043F0FF0E63EC2BF09BEF08F0120E295C60
:100FC000D8A402EF08F0FF0E63EC2BF059EC43F0CD
:100FD000FF0E63EC2BF0B9EC43F0FF0E63EC2BF04B
:100FE000A9EC43F0FF0E63EC2BF0BF0E63EC2BF08B
:100FF000FF0E63EC2BF089EC43F0FF0E63EC2BF05B
:101000009BEF08F0100E295CD8A426EF08F0000E24
:1010100063EC2BF0B9EC48F0000E63EC2BF0000E03
:1010200063EC2BF0FF0E63EC2BF059EC43F0FF0E5A
:1010300063EC2BF0D9EC43F0FF0E63EC2BF069EC82
:1010400043F0FF0E63EC2BF09BEF08F00F0E295CD2
:10105000D8A44AEF08F0000E63EC2BF0B9EC48F08E
:10106000000E63EC2BF0000E63EC2BF0FF0E63EC34
:101070002BF059EC43F0FF0E63EC2BF0D9EC43F06E
:10108000FF0E63EC2BF069EC43F0FF0E63EC2BF0EA
:101090009BEF08F0000E63EC2BF0100E63EC2BF0CE
:1010A000100E63EC2BF0100E63EC2BF0100E63ECC3
:1010B0002BF0100E63EC2BF0000E63EC2BF0100EF7
:1010C00063EC2BF0100E63EC2BF0100E63EC2BF0A6
:1010D000100E63EC2BF0100E63EC2BF0000E63ECA3
:1010E0002BF0100E63EC2BF0100E63EC2BF0100EB7
:1010F00063EC2BF0100E63EC2BF0100E63EC2BF076
:10110000000E63EC2BF0400E63EC2BF0000E63EC52
:101110002BF0100E63EC2BF0100E63EC2BF0100E86
:1011200063EC2BF0100E63EC2BF0100E63EC2BF045
:10113000000E63EC2BF0000E63EC2BF019EC46F084
:10114000000E63EC2BF0F9EC45F0000E63EC2BF095
:1011500009EC47F0000E63EC2BF025EC2BF0400E71
:1011600031EC2BF0BC0E4AEC2BF0000E63EC2BF0B4
:1011700009EC46F0000E63EC2BF049EC46F0000E53
:1011800063EC2BF0280E63EC2BF0280E63EC2BF0B5
:10119000280E63EC2BF0280E63EC2BF0280E63EC8A
:1011A0002BF0000E63EC2BF025EC2BF0530E31EC02
:1011B0002BF0BC0E4AEC2BF01550380B406E000E95
:1011C000405CD8A40CEF09F0000E63EC2BF089EC26
:1011D00046F0000E63EC2BF0E9EC46F0000E63ECF9
:1011E0002BF069EC46F0000E63EC2BF0A9EC42F01A
:1011F000000E63EC2BF0B9EC48F0000E63EC2BF022
:10120000B9EC48F0000E63EC2BF0B9EC48F0000E9E
:1012100063EC2BF057EF0AF0080E405CD8A439EFCE
:1012200009F0000E63EC2BF089EC46F0000E63EC45
:101230002BF0E9EC46F0000E63EC2BF069EC46F085
:10124000000E63EC2BF0B9EC42F0000E63EC2BF0D7
:10125000B9EC48F0000E63EC2BF0B9EC48F0000E4E
:1012600063EC2BF0B9EC48F0000E63EC2BF057EF79
:101270000AF0100E405CD8A466EF09F0000E63EC93
:101280002BF089EC46F0000E63EC2BF0E9EC46F015
:10129000000E63EC2BF069EC46F0000E63EC2BF0D3
:1012A000C9EC42F0000E63EC2BF0B9EC48F0000EF4
:1012B00063EC2BF0B9EC48F0000E63EC2BF0B9ECCA
:1012C00048F0000E63EC2BF057EF0AF0180E405C6C
:1012D000D8A4AAEF09F0000E63EC2BF0B9EC46F0AD
:1012E000000E63EC2BF099EC46F0000E63EC2BF053
:1012F00099EC45F0000E63EC2BF0B9EC48F083A2BA
:1013000096EF09F0FF0E63EC2BF019EC47F0FF0E9F
:1013100063EC2BF039EC47F0FF0E63EC2BF049EC5B
:1013200048F0FF0E63EC2BF057EF0AF0000E63EC71
:101330002BF099EC46F0000E63EC2BF069EC46F0D4
:10134000000E63EC2BF0B9EC45F0000E63EC2BF0D3
:1013500057EF0AF0200E405CD8A4D7EF09F0000E3A
:1013600063EC2BF089EC46F0000E63EC2BF0E9EC1B
:1013700046F0000E63EC2BF069EC46F0000E63ECD7
:101380002BF0E9EC42F0000E63EC2BF0B9EC48F0E6
:10139000000E63EC2BF0B9EC48F0000E63EC2BF080
:1013A000B9EC48F0000E63EC2BF057EF0AF0280E72
:1013B000405CD8A404EF0AF0000E63EC2BF089EC3B
:1013C00046F0000E63EC2BF0E9EC46F0000E63EC07
:1013D0002BF069EC46F0000E63EC2BF0F9EC42F0D8
:1013E000000E63EC2BF0B9EC48F0000E63EC2BF030
:1013F000B9EC48F0000E63EC2BF0B9EC48F0000EAD
:1014000063EC2BF057EF0AF0300E405CD8A431EFBC
:101410000AF0000E63EC2BF089EC46F0000E63EC52
:101420002BF0E9EC46F0000E63EC2BF069EC46F093
:10143000000E63EC2BF009EC43F0000E63EC2BF094
:10144000B9EC48F0000E63EC2BF0B9EC48F0000E5C
:1014500063EC2BF0B9EC48F0000E63EC2BF057EF87
:101460000AF0000E63EC2BF089EC46F0000E63EC02
:101470002BF0E9EC46F0000E63EC2BF069EC46F043
:10148000000E63EC2BF019EC43F0000E63EC2BF034
:10149000B9EC48F0000E63EC2BF0B9EC48F0000E0C
:1014A00063EC2BF0B9EC48F0000E63EC2BF01DA8B8
:1014B00050921DB872EF0AF0020E1F5CD8B47EEF96
:1014C0000AF0030E1F5CD8B47EEF0AF0010E1F5C19
:1014D000D8B47EEF0AF0210E1F5CD8B47EEF0AF07C
:1014E00078EF0AF050B278EF0AF06AEC2CF05082F4
:1014F000206A216A226A236A266A276A2050CEEC73
:1015000039F025EC2BF0400E31EC2BF0BE0E4AECFE
:101510002BF0080E63EC2BF0F80E63EC2BF0080EAA
:1015200063EC2BF0E00E63EC2BF0200E63EC2BF061
:10153000000E63EC2BF0000E63EC2BF0059CEAEC44
:1015400039F02150CEEC39F025EC2BF05A0E31EC6D
:101550002BF0BE0E4AEC2BF0F80E63EC2BF0000ED5
:1015600063EC2BF0E00E63EC2BF0200E63EC2BF021
:10157000E00E63EC2BF0000E63EC2BF0000E63EC3E
:101580002BF0059CEAEC39F02250CEEC39F025EC3A
:101590002BF0400E31EC2BF0BF0E4AEC2BF0059CEB
:1015A000EAEC39F0D9EC48F02350CEEC39F025ECD8
:1015B0002BF04E0E31EC2BF0BF0E4AEC2BF0059CBD
:1015C000EAEC39F02650CEEC39F025EC2BF05C0E2D
:1015D00031EC2BF0BF0E4AEC2BF0059CEAEC39F015
:1015E000D9EC48F02750CEEC39F025EC2BF06A0E00
:1015F00031EC2BF0BF0E4AEC2BF0059CEAEC39F0F5
:1016000028EC2BF0460E31EC2BF0BC0E4AEC2BF004
:10161000700E63EC2BF0100E63EC2BF0100E63ECED
:101620002BF0100E63EC2BF0000E63EC2BF0E9ECCA
:1016300045F0000E63EC2BF069EC46F0000E63EC15
:101640002BF059EC46F0000E63EC2BF0082A220E2A
:10165000085CD8B431EF0BF0100E63EC2BF026EFE2
:101660000BF0086A700E63EC2BF028EC2BF0460EA2
:1016700031EC2BF0BD0E4AEC2BF0000E63EC2BF09E
:10168000A9EC42F0000E63EC2BF0280E63EC2BF07B
:10169000280E63EC2BF0280E63EC2BF0280E63EC85
:1016A0002BF0280E63EC2BF0000E63EC2BF01350A4
:1016B0000F0B406EFFEC2EF028EC2BF0460E31ECB9
:1016C0002BF0BE0E4AEC2BF0000E63EC2BF0B9ECC5
:1016D00042F0000E63EC2BF0280E63EC2BF0280E8A
:1016E00063EC2BF0280E63EC2BF0280E63EC2BF050
:1016F000280E63EC2BF0000E63EC2BF01450F00B73
:10170000406E4042404240424042FFEC2EF028EC06
:101710002BF0460E31EC2BF0BF0E4AEC2BF0000EF6
:1017200063EC2BF0C9EC42F0000E63EC2BF0280EBA
:1017300063EC2BF0280E63EC2BF0280E63EC2BF0FF
:10174000280E63EC2BF0280E63EC2BF0000E63ECFC
:101750002BF014500F0B406EFFEC2EF023EF01F036
:101760004F6A25EC2BF0410E31EC2BF0B80E4AEC11
:101770002BF0700E63EC2BF0100E63EC2BF0100EC0
:1017800063EC2BF0100E63EC2BF0000E63EC2BF0EF
:10179000A9EC45F0000E63EC2BF099EC46F0000E3E
:1017A00063EC2BF029EC43F0000E63EC2BF0E9EC3A
:1017B00042F0000E63EC2BF0B9EC42F0000E63EC4B
:1017C0002BF009EC43F0000E63EC2BF0B9EC48F081
:1017D00089EC46F0000E63EC2BF0C9EC45F0000EEE
:1017E00063EC2BF0E9EC45F028EC2BF0400E31ECEB
:1017F0002BF0B80E4AEC2BF0000E63EC2BF009EC4A
:1018000046F0000E63EC2BF099EC46F0000E63EC12
:101810002BF0A9EC46F0000E63EC2BF0C9EC45F080
:10182000000E63EC2BF089EC46F0000E63EC2BF01D
:10183000082A200E085CD8B423EF0CF0100E63ECDD
:101840002BF018EF0CF0086A700E63EC2BF025EC0F
:101850002BF0410E31EC2BF0B90E4AEC2BF0FF0EC1
:1018600063EC2BF019EC47F0FF0E63EC2BF049EC26
:1018700047F0FF0E63EC2BF049EC47F0FF0E63ECF2
:101880002BF029EC48F0FF0E63EC2BF059EC47F0FD
:10189000FF0E63EC2BF039EC48F0FF0E63EC2BF0FD
:1018A00039EC48F0FF0E63EC2BF028EC2BF0410EE6
:1018B00031EC2BF0B90E4AEC2BF0FF0E63EC2BF061
:1018C00049EC47F0FF0E63EC2BF019EC47F0FF0EEC
:1018D00063EC2BF049EC48F0FF0E63EC2BF019ECB5
:1018E00047F0FF0E63EC2BF080B091EF0CF0070E89
:1018F000555CD8B47FEF0CF0552A93EF0CF0556A85
:101900003EB093EF0CF0060E425CD8B48BEF0CF0B7
:10191000422A8CEF0CF0426A4DEC2CF03E8093EFA3
:101920000CF03E90556A84B6B1EF0CF0070E545C93
:10193000D8B49EEF0CF0542AB3EF0CF0546A3EBCBE
:10194000B3EF0CF0000E425CD8B4AAEF0CF04206E4
:10195000ACEF0CF0060E426E4DEC2CF03E8CB3EF6B
:101960000CF03E9C546A25EC2BF0410E31EC2BF030
:10197000BA0E4AEC2BF0000E425CD8B4E0EF0CF04B
:10198000010E425CD8B4A6EF0DF0020E425CD8B452
:101990006CEF0EF0030E425CD8B432EF0FF0040E81
:1019A000425CD8B4F8EF0FF0050E425CD8B4BEEF3D
:1019B00010F0060E425CD8B484EF11F0E2EF11F0A3
:1019C000A9EC42F0000E63EC2BF0A9EC42F0000E03
:1019D00063EC2BF0F9EC45F0000E63EC2BF028ECF7
:1019E0002BF0410E31EC2BF0BA0E4AEC2BF01150DB
:1019F00028EC3AF025EC2BF0410E31EC2BF0BB0E2D
:101A00004AEC2BF0A9EC42F0000E63EC2BF0B9ECA1
:101A100042F0000E63EC2BF0F9EC45F0000E63ECA5
:101A20002BF028EC2BF0410E31EC2BF0BB0E4AECE6
:101A30002BF0125028EC3AF025EC2BF0410E31EC53
:101A40002BF0BC0E4AEC2BF0A9EC42F0000E63EC3C
:101A50002BF0C9EC42F0000E63EC2BF0F9EC45F0F2
:101A6000000E63EC2BF028EC2BF0410E31EC2BF048
:101A7000BC0E4AEC2BF0135028EC3AF025EC2BF07E
:101A8000410E31EC2BF0BD0E4AEC2BF0A9EC42F0EC
:101A9000000E63EC2BF0D9EC42F0000E63EC2BF05F
:101AA000F9EC45F0000E63EC2BF028EC2BF0410E26
:101AB00031EC2BF0BD0E4AEC2BF0145028EC3AF030
:101AC00025EC2BF0410E31EC2BF0BE0E4AEC2BF046
:101AD000A9EC42F0000E63EC2BF0E9EC42F0000EB2
:101AE00063EC2BF0F9EC45F0000E63EC2BF028ECE6
:101AF0002BF0410E31EC2BF0BE0E4AEC2BF01550C2
:101B000028EC3AF025EC2BF0410E31EC2BF0BF0E17
:101B10004AEC2BF0A9EC42F0000E63EC2BF0F9EC50
:101B200042F0000E63EC2BF0F9EC45F0000E63EC94
:101B30002BF028EC2BF0410E31EC2BF0BF0E4AECD1
:101B40002BF0165028EC3AF0E2EF11F0A9EC42F03D
:101B5000000E63EC2BF009EC43F0000E63EC2BF06D
:101B6000F9EC45F0000E63EC2BF028EC2BF0410E65
:101B700031EC2BF0BA0E4AEC2BF0175028EC3AF06F
:101B800025EC2BF0410E31EC2BF0BB0E4AEC2BF088
:101B9000A9EC42F0000E63EC2BF019EC43F0000EC0
:101BA00063EC2BF0F9EC45F0000E63EC2BF028EC25
:101BB0002BF0410E31EC2BF0BB0E4AEC2BF0185001
:101BC00028EC3AF025EC2BF0410E31EC2BF0BC0E5A
:101BD0004AEC2BF0A9EC42F0000E63EC2BF029EC60
:101BE00043F0000E63EC2BF0F9EC45F0000E63ECD3
:101BF0002BF028EC2BF0410E31EC2BF0BC0E4AEC14
:101C00002BF0195028EC3AF025EC2BF0410E31EC7A
:101C10002BF0BD0E4AEC2BF0A9EC42F0000E63EC69
:101C20002BF039EC43F0000E63EC2BF0F9EC45F0AF
:101C3000000E63EC2BF028EC2BF0410E31EC2BF076
:101C4000BD0E4AEC2BF01A5028EC3AF025EC2BF0A4
:101C5000410E31EC2BF0BE0E4AEC2BF0A9EC42F019
:101C6000000E63EC2BF089EC45F0000E63EC2BF0DA
:101C7000F9EC45F0000E63EC2BF028EC2BF0410E54
:101C800031EC2BF0BE0E4AEC2BF01B5028EC3AF056
:101C900025EC2BF0410E31EC2BF0BF0E4AEC2BF073
:101CA000A9EC42F0000E63EC2BF099EC45F0000E2D
:101CB00063EC2BF0F9EC45F0000E63EC2BF028EC14
:101CC0002BF0410E31EC2BF0BF0E4AEC2BF01C50E8
:101CD00028EC3AF0E2EF11F0A9EC42F0000E63ECD0
:101CE0002BF0A9EC45F0000E63EC2BF0F9EC45F07D
:101CF000000E63EC2BF028EC2BF0410E31EC2BF0B6
:101D0000BA0E4AEC2BF01D5028EC3AF025EC2BF0E3
:101D1000410E31EC2BF0BB0E4AEC2BF0A9EC42F05B
:101D2000000E63EC2BF0B9EC45F0000E63EC2BF0E9
:101D3000F9EC45F0000E63EC2BF028EC2BF0410E93
:101D400031EC2BF0BB0E4AEC2BF01E5028EC3AF095
:101D500025EC2BF0410E31EC2BF0BC0E4AEC2BF0B5
:101D6000A9EC42F0000E63EC2BF0C9EC45F0000E3C
:101D700063EC2BF0F9EC45F0000E63EC2BF028EC53
:101D80002BF0410E31EC2BF0BC0E4AEC2BF01F5027
:101D900028EC3AF025EC2BF0410E31EC2BF0BD0E87
:101DA0004AEC2BF0A9EC42F0000E63EC2BF0D9ECDE
:101DB00045F0000E63EC2BF0F9EC45F0000E63ECFF
:101DC0002BF028EC2BF0410E31EC2BF0BD0E4AEC41
:101DD0002BF0205028EC3AF025EC2BF0410E31ECA2
:101DE0002BF0BE0E4AEC2BF0B9EC42F0000E63EC87
:101DF0002BF0A9EC42F0000E63EC2BF0F9EC45F06F
:101E0000000E63EC2BF028EC2BF0410E31EC2BF0A4
:101E1000BE0E4AEC2BF0215028EC3AF025EC2BF0CA
:101E2000410E31EC2BF0BF0E4AEC2BF0B9EC42F036
:101E3000000E63EC2BF0B9EC42F0000E63EC2BF0DB
:101E4000F9EC45F0000E63EC2BF028EC2BF0410E82
:101E500031EC2BF0BF0E4AEC2BF0225028EC3AF07C
:101E6000E2EF11F0B9EC42F0000E63EC2BF0C9EC9C
:101E700042F0000E63EC2BF0F9EC45F0000E63EC41
:101E80002BF028EC2BF0410E31EC2BF0BA0E4AEC83
:101E90002BF0235028EC3AF025EC2BF0410E31ECDE
:101EA0002BF0BB0E4AEC2BF0B9EC42F0000E63ECC9
:101EB0002BF0D9EC42F0000E63EC2BF0F9EC45F07E
:101EC000000E63EC2BF028EC2BF0410E31EC2BF0E4
:101ED000BB0E4AEC2BF0245028EC3AF025EC2BF00A
:101EE000410E31EC2BF0BC0E4AEC2BF0B9EC42F079
:101EF000000E63EC2BF0E9EC42F0000E63EC2BF0EB
:101F0000F9EC45F0000E63EC2BF028EC2BF0410EC1
:101F100031EC2BF0BC0E4AEC2BF0255028EC3AF0BB
:101F200025EC2BF0410E31EC2BF0BD0E4AEC2BF0E2
:101F3000B9EC42F0000E63EC2BF0F9EC42F0000E2D
:101F400063EC2BF0F9EC45F0000E63EC2BF028EC81
:101F50002BF0410E31EC2BF0BD0E4AEC2BF026504D
:101F600028EC3AF025EC2BF0410E31EC2BF0BE0EB4
:101F70004AEC2BF0B9EC42F0000E63EC2BF009ECCC
:101F800043F0000E63EC2BF0F9EC45F0000E63EC2F
:101F90002BF028EC2BF0410E31EC2BF0BE0E4AEC6E
:101FA0002BF0275028EC3AF025EC2BF0410E31ECC9
:101FB0002BF0BF0E4AEC2BF0B9EC42F0000E63ECB4
:101FC0002BF019EC43F0000E63EC2BF0F9EC45F02C
:101FD000000E63EC2BF028EC2BF0410E31EC2BF0D3
:101FE000BF0E4AEC2BF0285028EC3AF0E2EF11F04B
:101FF000B9EC42F0000E63EC2BF029EC43F0000E3C
:1020000063EC2BF0F9EC45F0000E63EC2BF028ECC0
:102010002BF0410E31EC2BF0BA0E4AEC2BF029508C
:1020200028EC3AF025EC2BF0410E31EC2BF0BB0EF6
:102030004AEC2BF0B9EC42F0000E63EC2BF039ECDB
:1020400043F0000E63EC2BF0F9EC45F0000E63EC6E
:102050002BF028EC2BF0410E31EC2BF0BB0E4AECB0
:102060002BF02A5028EC3AF025EC2BF0410E31EC05
:102070002BF0BC0E4AEC2BF0B9EC42F0000E63ECF6
:102080002BF089EC45F0000E63EC2BF0F9EC45F0F9
:10209000000E63EC2BF028EC2BF0410E31EC2BF012
:1020A000BC0E4AEC2BF02B5028EC3AF025EC2BF030
:1020B000410E31EC2BF0BD0E4AEC2BF0B9EC42F0A6
:1020C000000E63EC2BF099EC45F0000E63EC2BF066
:1020D000F9EC45F0000E63EC2BF028EC2BF0410EF0
:1020E00031EC2BF0BD0E4AEC2BF02C5028EC3AF0E2
:1020F00025EC2BF0410E31EC2BF0BE0E4AEC2BF010
:10210000B9EC42F0000E63EC2BF0A9EC45F0000EA8
:1021100063EC2BF0F9EC45F0000E63EC2BF028ECAF
:102120002BF0410E31EC2BF0BE0E4AEC2BF02D5073
:1021300028EC3AF025EC2BF0410E31EC2BF0BF0EE1
:102140004AEC2BF0B9EC42F0000E63EC2BF0B9EC4A
:1021500045F0000E63EC2BF0F9EC45F0000E63EC5B
:102160002BF028EC2BF0410E31EC2BF0BF0E4AEC9B
:102170002BF02E5028EC3AF0E2EF11F0B9EC42F0DF
:10218000000E63EC2BF0C9EC45F0000E63EC2BF075
:10219000F9EC45F0000E63EC2BF028EC2BF0410E2F
:1021A00031EC2BF0BA0E4AEC2BF02F5028EC3AF021
:1021B00025EC2BF0410E31EC2BF0BB0E4AEC2BF052
:1021C000B9EC42F0000E63EC2BF0D9EC45F0000EB8
:1021D00063EC2BF0F9EC45F0000E63EC2BF028ECEF
:1021E0002BF0410E31EC2BF0BB0E4AEC2BF03050B3
:1021F00028EC3AF025EC2BF0410E31EC2BF0BC0E24
:102200004AEC2BF0C9EC42F0000E63EC2BF0A9EC89
:1022100042F0000E63EC2BF0F9EC45F0000E63EC9D
:102220002BF028EC2BF0410E31EC2BF0BC0E4AECDD
:102230002BF0315028EC3AF025EC2BF0410E31EC2C
:102240002BF0BD0E4AEC2BF0C9EC42F0000E63EC13
:102250002BF0B9EC42F0000E63EC2BF0F9EC45F0FA
:10226000000E63EC2BF028EC2BF0410E31EC2BF040
:10227000BD0E4AEC2BF0325028EC3AF025EC2BF056
:10228000410E31EC2BF0BE0E4AEC2BF0C9EC42F0C3
:10229000000E63EC2BF0C9EC42F0000E63EC2BF067
:1022A000F9EC45F0000E63EC2BF028EC2BF0410E1E
:1022B00031EC2BF0BE0E4AEC2BF0335028EC3AF008
:1022C00025EC2BF0410E31EC2BF0BF0E4AEC2BF03D
:1022D000C9EC42F0000E63EC2BF0D9EC42F0000E9A
:1022E00063EC2BF0F9EC45F0000E63EC2BF028ECDE
:1022F0002BF0410E31EC2BF0BF0E4AEC2BF034509A
:1023000028EC3AF0E2EF11F0C9EC42F0000E63EC79
:102310002BF0E9EC42F0000E63EC2BF0F9EC45F009
:10232000000E63EC2BF028EC2BF0410E31EC2BF07F
:10233000BA0E4AEC2BF0355028EC3AF025EC2BF095
:10234000410E31EC2BF0BB0E4AEC2BF0C9EC42F005
:10235000000E63EC2BF0F9EC42F0000E63EC2BF076
:10236000F9EC45F0000E63EC2BF028EC2BF0410E5D
:1023700031EC2BF0BB0E4AEC2BF0365028EC3AF047
:1023800025EC2BF0410E31EC2BF0BC0E4AEC2BF07F
:10239000C9EC42F0000E63EC2BF009EC43F0000EA8
:1023A00063EC2BF0F9EC45F0000E63EC2BF028EC1D
:1023B0002BF0410E31EC2BF0BC0E4AEC2BF03750D9
:1023C00028EC3AF0E6EC2EF023EF01F025EC2BF0B0
:1023D000410E31EC2BF0B80E4AEC2BF0700E63EC92
:1023E0002BF0100E63EC2BF0100E63EC2BF0100EA4
:1023F00063EC2BF0000E63EC2BF0A9EC45F0000E23
:1024000063EC2BF099EC46F0000E63EC2BF029EC1A
:1024100043F0000E63EC2BF0E9EC42F0000E63ECAD
:102420002BF0B9EC42F0000E63EC2BF009EC43F01A
:10243000000E63EC2BF0B9EC48F099EC46F0000E7E
:1024400063EC2BF0C9EC45F0000E63EC2BF0A9EC2B
:1024500046F028EC2BF0400E31EC2BF0B80E4AEC95
:102460002BF0000E63EC2BF0A9EC46F0000E63ECB1
:102470002BF009EC46F0000E63EC2BF049EC46F033
:10248000000E63EC2BF0E9EC45F0000E63EC2BF052
:10249000082A260E085CD8B453EF12F0100E63EC35
:1024A0002BF048EF12F0086A700E63EC2BF0000E70
:1024B000435CD8B463EF12F0010E435CD8B4A3EFD1
:1024C00015F023EF01F025EC2BF0460E31EC2BF04C
:1024D000B90E4AEC2BF099EC46F0000E63EC2BF0B1
:1024E000C9EC45F0000E63EC2BF029EC46F0000E31
:1024F00063EC2BF0C9EC45F0000E63EC2BF0A9EC7B
:1025000045F0000E63EC2BF0A9EC46F0000E63ECF6
:102510002BF0B9EC48F089EC45F0000E63EC2BF0A1
:10252000B9EC45F0000E63EC2BF0B9EC45F028EC6B
:102530002BF0400E31EC2BF0B90E4AEC2BF0000ED4
:1025400063EC2BF089EC46F0000E63EC2BF0C9EC49
:1025500045F0000E63EC2BF099EC46F0000E63ECB6
:102560002BF099EC46F0000E63EC2BF080B0D1EF2D
:1025700012F0070E555CD8B4C1EF12F0552AD3EF14
:1025800012F0556A3EB0D3EF12F00A0E465CD8B492
:10259000CDEF12F0462ACEEF12F0466A3E80D3EF1E
:1025A00012F03E90556A84B6EFEF12F0070E545CBD
:1025B000D8B4DEEF12F0542AF1EF12F0546A3EBCA8
:1025C000F1EF12F0000E465CD8B4EAEF12F04606C6
:1025D000ECEF12F00A0E466E3E8CF1EF12F03E9CCC
:1025E000546A3F9425EC2BF04A0E31EC2BF0BB0ED5
:1025F0004AEC2BF0000E465CD8B413EF13F0000E3B
:1026000063EC2BF0A9EC42F0000E63EC2BF0A9EC8C
:1026100042F0000E63EC2BF0F9EC45F0000E63EC99
:102620002BF025EF13F0FF0E63EC2BF049EC43F099
:10263000FF0E63EC2BF049EC43F0FF0E63EC2BF044
:1026400089EC47F0FF0E63EC2BF025EC2BF0670EC6
:1026500031EC2BF0BB0E4AEC2BF0010E465CD8B4EB
:1026600046EF13F0000E63EC2BF0A9EC42F0000EE5
:1026700063EC2BF0B9EC42F0000E63EC2BF0F9ECBC
:1026800045F0000E63EC2BF058EF13F0FF0E63ECF7
:102690002BF049EC43F0FF0E63EC2BF059EC43F0C8
:1026A000FF0E63EC2BF089EC47F0FF0E63EC2BF090
:1026B00028EC2BF0440E31EC2BF0BB0E4AEC2BF047
:1026C000020E465CD8B479EF13F0000E63EC2BF0E9
:1026D000A9EC42F0000E63EC2BF0C9EC42F0000EC6
:1026E00063EC2BF0F9EC45F0000E63EC2BF08BEF74
:1026F00013F0FF0E63EC2BF049EC43F0FF0E63EC9C
:102700002BF069EC43F0FF0E63EC2BF089EC47F003
:10271000FF0E63EC2BF028EC2BF0610E31EC2BF06C
:10272000BB0E4AEC2BF0030E465CD8B4ACEF13F0B2
:10273000000E63EC2BF0A9EC42F0000E63EC2BF0E2
:10274000D9EC42F0000E63EC2BF0F9EC45F0000EF2
:1027500063EC2BF0BEEF13F0FF0E63EC2BF049ECB3
:1027600043F0FF0E63EC2BF079EC43F0FF0E63ECCB
:102770002BF089EC47F0FF0E63EC2BF025EC2BF0EF
:102780004A0E31EC2BF0BC0E4AEC2BF0040E465CEA
:10279000D8B4DFEF13F0000E63EC2BF0A9EC42F09D
:1027A000000E63EC2BF0E9EC42F0000E63EC2BF032
:1027B000F9EC45F0000E63EC2BF0F1EF13F0FF0E97
:1027C00063EC2BF049EC43F0FF0E63EC2BF089EC4B
:1027D00043F0FF0E63EC2BF089EC47F0FF0E63EC47
:1027E0002BF025EC2BF0670E31EC2BF0BC0E4AECF5
:1027F0002BF0050E465CD8B412EF14F0000E63EC1B
:102800002BF0A9EC42F0000E63EC2BF0F9EC42F057
:10281000000E63EC2BF0F9EC45F0000E63EC2BF0AE
:1028200024EF14F0FF0E63EC2BF049EC43F0FF0EA5
:1028300063EC2BF099EC43F0FF0E63EC2BF089EC8A
:1028400047F0FF0E63EC2BF028EC2BF0440E31EC3C
:102850002BF0BC0E4AEC2BF0060E465CD8B445EFCC
:1028600014F0000E63EC2BF0A9EC42F0000E63ECC8
:102870002BF009EC43F0000E63EC2BF0F9EC45F083
:10288000000E63EC2BF057EF14F0FF0E63EC2BF00F
:1028900049EC43F0FF0E63EC2BF0A9EC43F0FF0E84
:1028A00063EC2BF089EC47F0FF0E63EC2BF028EC87
:1028B0002BF0610E31EC2BF0B40E4AEC2BF0070E2E
:1028C000465CD8B478EF14F0000E63EC2BF0A9EC62
:1028D00042F0000E63EC2BF019EC43F0000E63ECB9
:1028E0002BF0F9EC45F0000E63EC2BF08AEF14F0BE
:1028F000FF0E63EC2BF049EC43F0FF0E63EC2BF082
:10290000B9EC43F0FF0E63EC2BF089EC47F0FF0EBF
:1029100063EC2BF025EC2BF04A0E31EC2BF0BD0EC6
:102920004AEC2BF0080E465CD8B4ABEF14F0000E66
:1029300063EC2BF0A9EC42F0000E63EC2BF029ECD9
:1029400043F0000E63EC2BF0F9EC45F0000E63EC65
:102950002BF0BDEF14F0FF0E63EC2BF049EC43F0CD
:10296000FF0E63EC2BF0C9EC43F0FF0E63EC2BF091
:1029700089EC47F0FF0E63EC2BF025EC2BF0670E93
:1029800031EC2BF0BD0E4AEC2BF0090E465CD8B4AE
:10299000DEEF14F0000E63EC2BF0A9EC42F0000E19
:1029A00063EC2BF039EC43F0000E63EC2BF0F9EC08
:1029B00045F0000E63EC2BF0F0EF14F0FF0E63EC2B
:1029C0002BF049EC43F0FF0E63EC2BF0D9EC43F015
:1029D000FF0E63EC2BF089EC47F0FF0E63EC2BF05D
:1029E00025EC2BF04A0E31EC2BF0BF0E4AEC2BF00D
:1029F0000A0E465CD8B443EF15F0000E63EC2BF0E2
:102A0000B9EC45F0000E63EC2BF0C9EC45F0000E7C
:102A100063EC2BF0D9EC45F0000E63EC2BF089EC65
:102A200045F0000E63EC2BF0B9EC46F0000E63ECC1
:102A30002BF029EC46F0000E63EC2BF0A9EC46F0ED
:102A4000000E63EC2BF0B9EC48F029EC46F0000ED8
:102A500063EC2BF028EC2BF0400E31EC2BF0BF0E8A
:102A60004AEC2BF059EC46F0000E63EC2BF089ECAD
:102A700045F0000E63EC2BF0B9EC45F0000E63EC72
:102A80002BF087EF15F0FF0E63EC2BF049EC47F0CD
:102A9000FF0E63EC2BF059EC47F0FF0E63EC2BF0CC
:102AA00069EC47F0FF0E63EC2BF019EC47F0FF0EDA
:102AB00063EC2BF059EC48F0FF0E63EC2BF0C9EC03
:102AC00047F0FF0E63EC2BF049EC48F0FF0E63EC8F
:102AD0002BF0C9EC48F0C9EC47F0FF0E63EC2BF08B
:102AE00028EC2BF0400E31EC2BF0BF0E4AEC2BF013
:102AF000F9EC47F0FF0E63EC2BF019EC47F0FF0EFA
:102B000063EC2BF049EC47F0FF0E63EC2BF0E6ECA6
:102B10002EF080B89FEF15F0070E575CD8B494EFF5
:102B200015F0572AA1EF15F0576A3EB8A1EF15F03E
:102B3000010E436E4DEC2CF03E88A1EF15F03E984F
:102B4000576A23EF01F025EC2BF0460E31EC2BF009
:102B5000B90E4AEC2BF0000E465CD8B4DFEF15F04E
:102B6000010E465CD8B4E0EF16F0020E465CD8B415
:102B700039EF18F0030E465CD8B44DEF19F0040E8F
:102B8000465CD8B431EF1AF0050E465CD8B440EF7D
:102B90001BF0060E465CD8B467EF1CF0070E465CCF
:102BA000D8B4CBEF1DF0080E465CD8B483EF1EF00E
:102BB000090E465CD8B43BEF1FF0F3EF1FF0F6ECC4
:102BC0003CF03FB2E6EF15F0050E496E3FB449EF19
:102BD00016F080B017EF16F0070E555CD8B4F4EF7E
:102BE00015F0552A19EF16F0556A3EB019EF16F098
:102BF000010E495CD8A401EF16F0080E496E14EFDF
:102C000016F0040E495CD8A40AEF16F0010E496EC6
:102C100014EF16F0080E495CD8A413EF16F0050E59
:102C2000496E14EF16F049063E8019EF16F03E90FB
:102C3000556A84B647EF16F0070E545CD8B424EFFB
:102C400016F0542A49EF16F0546A3EBC49EF16F0CC
:102C5000080E495CD8A431EF16F0010E496E44EF1E
:102C600016F0010E495CD8A43AEF16F0040E496E36
:102C700044EF16F0050E495CD8A443EF16F0080E99
:102C8000496E44EF16F0492A3E8C49EF16F03E9CFF
:102C9000546A25EC2BF0460E31EC2BF0BC0E4AECBE
:102CA0002BF0010E495CD8B483EF16F0040E495C9A
:102CB000D8B4A6EF16F0080E495CD8B4C7EF16F0EA
:102CC000FF0E63EC2BF049EC48F0FF0E63EC2BF0A9
:102CD00029EC48F0FF0E63EC2BF059EC48F0FF0EA6
:102CE00063EC2BF0E9EC47F0FF0E63EC2BF039ECD2
:102CF00047F0FF0E63EC2BF0B9EC48F0000E63ECEC
:102D00002BF0C7EF16F0FF0E63EC2BF069EC47F0E9
:102D1000FF0E63EC2BF039EC48F0FF0E63EC2BF068
:102D200079EC48F0FF0E63EC2BF039EC47F0FF0E26
:102D300063EC2BF0C9EC47F0FF0E63EC2BF0B9EC21
:102D400047F0FF0E63EC2BF0C7EF16F0FF0E63ECBD
:102D50002BF009EC48F0FF0E63EC2BF049EC47F048
:102D6000FF0E63EC2BF059EC48F0FF0E63EC2BF0F8
:102D700029EC48F0FF0E63EC2BF0B9EC48F0000EA4
:102D800063EC2BF0B9EC48F0000E63EC2BF03FB68F
:102D9000CEEF16F03F8611504A6E4B6E94EC32F037
:102DA00028EC2BF0400E31EC2BF0BD0E4AEC2BF052
:102DB000405040EC3AF089EC3AF03F82FEEF20F0D0
:102DC0004FEC3DF03FB2E7EF16F0070E496E3FA41F
:102DD0001AEC32F025EC2BF0460E31EC2BF0BC0E49
:102DE0004AEC2BF0000E495CD8B442EF17F0010E0C
:102DF000495CD8B46AEF17F0020E495CD8B492EF80
:102E000017F0030E495CD8B492EF17F0040E495C3A
:102E1000D8B4C6EF17F0050E495CD8B4C6EF17F06A
:102E2000060E495CD8B4FAEF17F0080E495CD8B426
:102E300020EF18F0FF0E63EC2BF039EC47F0FF0E9B
:102E400063EC2BF089EC47F0FF0E63EC2BF039ECD0
:102E500048F0FF0E63EC2BF0B9EC48F0000E63EC89
:102E60002BF0B9EC48F0000E63EC2BF0B9EC48F015
:102E7000000E63EC2BF0B9EC48F0000E63EC2BF085
:102E800020EF18F0FF0E63EC2BF039EC48F0FF0E4A
:102E900063EC2BF079EC48F0FF0E63EC2BF039EC8F
:102EA00047F0FF0E63EC2BF0C9EC47F0FF0E63EC2C
:102EB0002BF0B9EC47F0FF0E63EC2BF0B9EC48F0C7
:102EC000000E63EC2BF0B9EC48F0000E63EC2BF035
:102ED00020EF18F0FF0E63EC2BF0D9EC47F0FF0E5B
:102EE00063EC2BF059EC48F0FF0E63EC2BF049EC4F
:102EF00048F0FF0E63EC2BF059EC47F0FF0E63EC4B
:102F00002BF039EC48F0FF0E63EC2BF019EC47F096
:102F1000FF0E63EC2BF0F9EC47F0FF0E63EC2BF0A7
:102F200020EF18F0FF0E63EC2BF099EC47F0FF0E4A
:102F300063EC2BF0E9EC47F0FF0E63EC2BF049EC6F
:102F400048F0FF0E63EC2BF0020E495CD8B4B0EFF2
:102F500017F049EC43F0FF0E63EC2BF0B5EF17F0E0
:102F600059EC43F0FF0E63EC2BF0B9EC48F0000E87
:102F700063EC2BF0B9EC48F0000E63EC2BF0B9ECED
:102F800048F0000E63EC2BF020EF18F0FF0E63EC1E
:102F90002BF089EC47F0FF0E63EC2BF0F9EC47F0D7
:102FA000FF0E63EC2BF0C9EC47F0FF0E63EC2BF047
:102FB00049EC47F0FF0E63EC2BF0040E495CD8B4EB
:102FC000E9EF17F049EC43F0FF0E63EC2BF0EEEF66
:102FD00017F059EC43F0FF0E63EC2BF0B9EC48F01E
:102FE000000E63EC2BF0B9EC48F0000E63EC2BF014
:102FF00020EF18F0FF0E63EC2BF029EC48F0FF0EE9
:1030000063EC2BF0D9EC47F0FF0E63EC2BF039ECBE
:1030100047F0FF0E63EC2BF0B9EC47F0FF0E63ECCA
:103020002BF069EC47F0FF0E63EC2BF0B9EC48F0A5
:10303000000E63EC2BF0B9EC48F0000E63EC2BF0C3
:103040003FB627EF18F03F8612504A6E4B6E94EC55
:1030500032F028EC2BF0400E31EC2BF0BD0E4AEC98
:103060002BF0405040EC3AF089EC3AF03F82FEEF12
:1030700020F0A8EC3DF03FB240EF18F0070E496E8B
:103080003FA41AEC32F025EC2BF0460E31EC2BF07D
:10309000BC0E4AEC2BF0000E495CD8B4BAEF18F025
:1030A000010E495CD8B4ECEF18F0020E495CD8B4BC
:1030B000ECEF18F0030E495CD8B4ECEF18F0080EF2
:1030C000495CD8B434EF19F0FF0E63EC2BF079ECC7
:1030D00047F0FF0E63EC2BF009EC48F0FF0E63ECB9
:1030E0002BF0F9EC47F0FF0E63EC2BF049EC43F0CA
:1030F000FF0E63EC2BF039EC48F0FF0E63EC2BF085
:1031000059EC47F0FF0E63EC2BF0C9EC47F0FF0ED3
:1031100063EC2BF0040E495CD8B4A0EF18F0050E58
:10312000495CD8B4A7EF18F0060E495CD8B4AEEFEE
:1031300018F049EC43F0FF0E63EC2BF0B3EF18F0FE
:1031400079EC43F0FF0E63EC2BF0B3EF18F069EC71
:1031500043F0FF0E63EC2BF0B3EF18F059EC43F0A3
:10316000FF0E63EC2BF0B9EC48F0000E63EC2BF093
:1031700034EF19F0FF0E63EC2BF049EC47F0FF0E33
:1031800063EC2BF059EC47F0FF0E63EC2BF049ECAD
:1031900048F0FF0E63EC2BF039EC47F0FF0E63ECC8
:1031A0002BF099EC47F0FF0E63EC2BF0B9EC48F0F4
:1031B000000E63EC2BF0B9EC48F0000E63EC2BF042
:1031C000B9EC48F0000E63EC2BF0B9EC48F0000EBF
:1031D00063EC2BF034EF19F0FF0E63EC2BF059EC9D
:1031E00047F0FF0E63EC2BF0D9EC47F0FF0E63ECD9
:1031F0002BF009EC48F0FF0E63EC2BF089EC47F064
:10320000FF0E63EC2BF039EC47F0FF0E63EC2BF074
:10321000E9EC47F0FF0E63EC2BF049EC48F0FF0EB1
:1032200063EC2BF0C9EC47F0FF0E63EC2BF0010EC2
:10323000495CD8B428EF19F0020E495CD8B42FEFDE
:1032400019F049EC43F0FF0E63EC2BF034EF19F06A
:1032500069EC43F0FF0E63EC2BF034EF19F059ECFE
:1032600043F0FF0E63EC2BF03FB63BEF19F03F86C7
:1032700013504A6E4B6E94EC32F028EC2BF0400E5B
:1032800031EC2BF0BD0E4AEC2BF0405040EC3AF004
:1032900089EC3AF03F82FEEF20F001EC3EF03FB2C5
:1032A00054EF19F0070E496E3FA41AEC32F025ECEA
:1032B0002BF0460E31EC2BF0BC0E4AEC2BF0000E3E
:1032C000495CD8B4C9EF19F0010E495CD8B4C9EF14
:1032D00019F0020E495CD8B4C9EF19F0030E495C2D
:1032E000D8B4C9EF19F0080E495CD8B418EF1AF039
:1032F000FF0E63EC2BF079EC47F0FF0E63EC2BF044
:1033000009EC48F0FF0E63EC2BF0F9EC47F0FF0EF0
:1033100063EC2BF069EC43F0FF0E63EC2BF039EC1F
:1033200048F0FF0E63EC2BF059EC47F0FF0E63EC16
:103330002BF0C9EC47F0FF0E63EC2BF0040E495C58
:10334000D8B4B4EF19F0050E495CD8B4BBEF19F04E
:10335000060E495CD8B4C2EF19F049EC43F0FF0EF9
:1033600063EC2BF018EF1AF079EC43F0FF0E63ECEE
:103370002BF018EF1AF069EC43F0FF0E63EC2BF022
:1033800018EF1AF059EC43F0FF0E63EC2BF018EF36
:103390001AF0FF0E63EC2BF079EC47F0FF0E63ECB4
:1033A0002BF009EC48F0FF0E63EC2BF0F9EC47F042
:1033B000FF0E63EC2BF059EC43F0FF0E63EC2BF0A7
:1033C00039EC48F0FF0E63EC2BF059EC47F0FF0EA0
:1033D00063EC2BF0C9EC47F0FF0E63EC2BF0000E12
:1033E000495CD8B405EF1AF0010E495CD8B40CEF73
:1033F0001AF0020E495CD8B413EF1AF049EC43F00E
:10340000FF0E63EC2BF018EF1AF079EC43F0FF0E8F
:1034100063EC2BF018EF1AF069EC43F0FF0E63EC4D
:103420002BF018EF1AF059EC43F0FF0E63EC2BF081
:103430003FB61FEF1AF03F8614504A6E4B6E94EC65
:1034400032F028EC2BF0400E31EC2BF0BD0E4AECA4
:103450002BF0405040EC3AF089EC3AF03F82FEEF1E
:1034600020F05AEC3EF03FB238EF1AF0070E496EEA
:103470003FA41AEC32F025EC2BF0460E31EC2BF089
:10348000BC0E4AEC2BF0000E495CD8B46DEF1AF07C
:10349000010E495CD8B490EF1AF0020E495CD8B422
:1034A000B3EF1AF0030E495CD8B4B3EF1AF0040E70
:1034B000495CD8B4B3EF1AF0050E495CD8B4EEEF0E
:1034C0001AF0060E495CD8B4EEEF1AF0080E495C0B
:1034D000D8B427EF1BF0EEEF1AF0FF0E63EC2BF0E1
:1034E00029EC48F0FF0E63EC2BF059EC48F0FF0E8E
:1034F00063EC2BF0E9EC47F0FF0E63EC2BF0B9EC3A
:1035000048F0000E63EC2BF0B9EC48F0000E63ECD1
:103510002BF0B9EC48F0000E63EC2BF027EF1BF01A
:10352000FF0E63EC2BF029EC48F0FF0E63EC2BF060
:1035300089EC48F0FF0E63EC2BF049EC47F0FF0EEE
:1035400063EC2BF0B9EC48F0000E63EC2BF0B9EC17
:1035500048F0000E63EC2BF0B9EC48F0000E63EC81
:103560002BF027EF1BF0FF0E63EC2BF029EC48F05B
:10357000FF0E63EC2BF089EC48F0FF0E63EC2BF0B0
:1035800039EC48F0FF0E63EC2BF059EC47F0FF0EDE
:1035900063EC2BF0C9EC47F0FF0E63EC2BF0020E4E
:1035A000495CD8B4E0EF1AF0030E495CD8B4E7EFF9
:1035B0001AF049EC43F0FF0E63EC2BF027EF1BF001
:1035C00069EC43F0FF0E63EC2BF027EF1BF059EC96
:1035D00043F0FF0E63EC2BF027EF1BF0FF0E63ECC4
:1035E0002BF049EC48F0FF0E63EC2BF089EC48F02F
:1035F000FF0E63EC2BF039EC48F0FF0E63EC2BF080
:1036000059EC47F0FF0E63EC2BF0C9EC47F0FF0ECE
:1036100063EC2BF0050E495CD8B41BEF1BF0060ED3
:10362000495CD8B422EF1BF049EC43F0FF0E63EC89
:103630002BF027EF1BF069EC43F0FF0E63EC2BF04F
:1036400027EF1BF059EC43F0FF0E63EC2BF03FB675
:103650002EEF1BF03F8615504A6E4B6E94EC32F005
:1036600028EC2BF0400E31EC2BF0BD0E4AEC2BF089
:10367000405040EC3AF089EC3AF03F82FEEF20F007
:10368000B3EC3EF03FB247EF1BF0070E496E3FA48C
:103690001AEC32F025EC2BF0460E31EC2BF0BC0E80
:1036A0004AEC2BF0080E495CD8B44EEF1CF0FF0E2C
:1036B00063EC2BF039EC48F0FF0E63EC2BF0F9ECE7
:1036C00047F0FF0E63EC2BF0000E495CD8B4A2EF7C
:1036D0001BF0010E495CD8B4BDEF1BF0020E495C33
:1036E000D8B4D8EF1BF0030E495CD8B4D8EF1BF068
:1036F000040E495CD8B4FFEF1BF0050E495CD8B44A
:103700001AEF1CF0060E495CD8B435EF1CF0C9EC7A
:1037100047F0FF0E63EC2BF029EC48F0FF0E63EC52
:103720002BF009EC48F0FF0E63EC2BF0F9EC47F0BE
:10373000FF0E63EC2BF0C9EC47F0FF0E63EC2BF0AF
:103740004EEF1CF0D9EC47F0FF0E63EC2BF039EC98
:1037500048F0FF0E63EC2BF0B9EC48F0000E63EC80
:103760002BF0B9EC48F0000E63EC2BF0B9EC48F00C
:10377000000E63EC2BF04EEF1CF039EC48F0FF0E1E
:1037800063EC2BF069EC47F0FF0E63EC2BF0B9EC27
:1037900048F0000E63EC2BF0B9EC48F0000E63EC3F
:1037A0002BF0B9EC48F0000E63EC2BF04EEF1CF060
:1037B00029EC48F0FF0E63EC2BF059EC47F0FF0EBC
:1037C00063EC2BF039EC48F0FF0E63EC2BF0020EAB
:1037D000495CD8B4F3EF1BF049EC43F0FF0E63EC07
:1037E0002BF0F8EF1BF059EC43F0FF0E63EC2BF0DD
:1037F000B9EC48F0000E63EC2BF04EEF1CF0A9EC96
:1038000047F0FF0E63EC2BF059EC48F0FF0E63EC31
:103810002BF039EC48F0FF0E63EC2BF049EC48F04C
:10382000FF0E63EC2BF0B9EC48F0000E63EC2BF0CC
:103830004EEF1CF049EC47F0FF0E63EC2BF059EC17
:1038400047F0FF0E63EC2BF0C9EC47F0FF0E63EC82
:103850002BF0B9EC48F0000E63EC2BF0B9EC48F01B
:10386000000E63EC2BF04EEF1CF039EC48F0FF0E2D
:1038700063EC2BF009EC48F0FF0E63EC2BF0F9EC55
:1038800047F0FF0E63EC2BF0C9EC47F0FF0E63EC42
:103890002BF0B9EC48F0000E63EC2BF03FB655EF7F
:1038A0001CF03F8616504A6E4B6E94EC32F028ECBA
:1038B0002BF0400E31EC2BF0BD0E4AEC2BF04050BB
:1038C00040EC3AF089EC3AF03F82FEEF20F05CECFD
:1038D0003FF03FB26EEF1CF0070E496E3FA457EC6D
:1038E00032F025EC2BF0460E31EC2BF0BC0E4AECFE
:1038F0002BF0010E495CD8B4C4EF1CF0020E495CF9
:10390000D8B4ECEF1CF0030E495CD8B414EF1DF0F2
:10391000040E495CD8B43CEF1DF0050E495CD8B4E8
:1039200064EF1DF0060E495CD8B48CEF1DF0080E54
:10393000495CD8B4B2EF1DF0FF0E63EC2BF009EC3C
:1039400048F0FF0E63EC2BF019EC47F0FF0E63EC30
:103950002BF029EC48F0FF0E63EC2BF0D9EC47F08C
:10396000FF0E63EC2BF0B9EC48F0000E63EC2BF08B
:10397000B9EC48F0000E63EC2BF0B9EC48F0000E07
:1039800063EC2BF0B2EF1DF0FF0E63EC2BF019ECA3
:1039900048F0FF0E63EC2BF039EC47F0FF0E63ECC0
:1039A0002BF029EC48F0FF0E63EC2BF039EC47F0DC
:1039B000FF0E63EC2BF0D9EC47F0FF0E63EC2BF01D
:1039C000B9EC48F0000E63EC2BF0B9EC48F0000EB7
:1039D00063EC2BF0B2EF1DF0FF0E63EC2BF039EC33
:1039E00047F0FF0E63EC2BF039EC47F0FF0E63EC71
:1039F0002BF029EC48F0FF0E63EC2BF039EC47F08C
:103A0000FF0E63EC2BF0D9EC47F0FF0E63EC2BF0CC
:103A1000B9EC48F0000E63EC2BF0B9EC48F0000E66
:103A200063EC2BF0B2EF1DF0FF0E63EC2BF059ECC2
:103A300048F0FF0E63EC2BF0E9EC47F0FF0E63EC6F
:103A40002BF0C9EC47F0FF0E63EC2BF0F9EC47F0DC
:103A5000FF0E63EC2BF039EC47F0FF0E63EC2BF01C
:103A6000B9EC47F0FF0E63EC2BF0D9EC47F0FF0EFA
:103A700063EC2BF0B2EF1DF0FF0E63EC2BF069EC62
:103A800048F0FF0E63EC2BF0D9EC47F0FF0E63EC2F
:103A90002BF0B9EC48F0000E63EC2BF0B9EC48F0D9
:103AA000000E63EC2BF0B9EC48F0000E63EC2BF049
:103AB000B9EC48F0000E63EC2BF0B9EC48F0000EC6
:103AC00063EC2BF0B2EF1DF0FF0E63EC2BF039EC42
:103AD00047F0FF0E63EC2BF0F9EC47F0FF0E63ECC0
:103AE0002BF0D9EC47F0FF0E63EC2BF069EC47F0BC
:103AF000FF0E63EC2BF0D9EC47F0FF0E63EC2BF0DC
:103B0000B9EC48F0000E63EC2BF0B9EC48F0000E75
:103B100063EC2BF0B2EF1DF0FF0E63EC2BF029EC01
:103B200047F0FF0E63EC2BF099EC47F0FF0E63ECCF
:103B30002BF009EC48F0FF0E63EC2BF0D9EC47F0CA
:103B4000FF0E63EC2BF0B9EC48F0000E63EC2BF0A9
:103B5000B9EC48F0000E63EC2BF0B9EC48F0000E25
:103B600063EC2BF03FB6B9EF1DF03F8617504A6E5D
:103B70004B6E94EC32F028EC2BF0400E31EC2BF035
:103B8000BD0E4AEC2BF0405040EC3AF089EC3AF094
:103B90003F82FEEF20F0EAEC3FF03FB2D2EF1DF0A3
:103BA000070E496E3FA457EC32F025EC2BF0460E81
:103BB00031EC2BF0BC0E4AEC2BF0010E495CD8B472
:103BC00013EF1EF0020E495CD8B421EF1EF0030E75
:103BD000495CD8B42AEF1EF0040E495CD8B438EF23
:103BE0001EF0050E495CD8B44BEF1EF0060E495C82
:103BF000D8B459EF1EF0080E495CD8B46AEF1EF035
:103C0000F6EC41F0D9EC47F0FF0E63EC2BF0B9EC89
:103C100048F0000E63EC2BF0B9EC48F0000E63ECBA
:103C20002BF06AEF1EF06BEC41F0D9EC47F0FF0E81
:103C300063EC2BF0B9EC48F0000E63EC2BF06AEF6C
:103C40001EF083EC41F0D9EC47F0FF0E63EC2BF053
:103C50006AEF1EF0A0EC41F0D9EC47F0FF0E63ECE8
:103C60002BF0B9EC48F0000E63EC2BF06AEF1EF07D
:103C7000B8EC41F0D9EC47F0FF0E63EC2BF0B9EC57
:103C800048F0000E63EC2BF0B9EC48F0000E63EC4A
:103C90002BF06AEF1EF0CBEC41F0D9EC47F0FF0EB1
:103CA00063EC2BF0B9EC48F0000E63EC2BF06AEFFC
:103CB0001EF0E3EC41F0D9EC47F0FF0E63EC2BF083
:103CC000B9EC48F0000E63EC2BF0B9EC48F0000EB4
:103CD00063EC2BF03FB671EF1EF03F8618504A6E32
:103CE0004B6E94EC32F028EC2BF0400E31EC2BF0C4
:103CF000BD0E4AEC2BF0405040EC3AF089EC3AF023
:103D00003F82FEEF20F059EC40F03FB28AEF1EF008
:103D1000070E496E3FA457EC32F025EC2BF0460E0F
:103D200031EC2BF0BC0E4AEC2BF0010E495CD8B400
:103D3000CBEF1EF0020E495CD8B4D9EF1EF0030E93
:103D4000495CD8B4E2EF1EF0040E495CD8B4F0EF41
:103D50001EF0050E495CD8B403EF1FF0060E495C57
:103D6000D8B411EF1FF0080E495CD8B422EF1FF051
:103D7000F6EC41F059EC43F0FF0E63EC2BF0B9EC9C
:103D800048F0000E63EC2BF0B9EC48F0000E63EC49
:103D90002BF022EF1FF06BEC41F059EC43F0FF0EDB
:103DA00063EC2BF0B9EC48F0000E63EC2BF022EF43
:103DB0001FF083EC41F059EC43F0FF0E63EC2BF065
:103DC00022EF1FF0A0EC41F059EC43F0FF0E63EC42
:103DD0002BF0B9EC48F0000E63EC2BF022EF1FF053
:103DE000B8EC41F059EC43F0FF0E63EC2BF0B9EC6A
:103DF00048F0000E63EC2BF0B9EC48F0000E63ECD9
:103E00002BF022EF1FF0CBEC41F059EC43F0FF0E0A
:103E100063EC2BF0B9EC48F0000E63EC2BF022EFD2
:103E20001FF0E3EC41F059EC43F0FF0E63EC2BF094
:103E3000B9EC48F0000E63EC2BF0B9EC48F0000E42
:103E400063EC2BF03FB629EF1FF03F8619504A6E06
:103E50004B6E94EC32F028EC2BF0400E31EC2BF052
:103E6000BD0E4AEC2BF0405040EC3AF089EC3AF0B1
:103E70003F82FEEF20F0E2EC40F03FB242EF1FF055
:103E8000070E496E3FA457EC32F025EC2BF0460E9E
:103E900031EC2BF0BC0E4AEC2BF0010E495CD8B48F
:103EA00083EF1FF0020E495CD8B491EF1FF0030EB0
:103EB000495CD8B49AEF1FF0040E495CD8B4A8EF5F
:103EC0001FF0050E495CD8B4BBEF1FF0060E495C2D
:103ED000D8B4C9EF1FF0080E495CD8B4DAEF1FF070
:103EE000F6EC41F049EC43F0FF0E63EC2BF0B9EC3B
:103EF00048F0000E63EC2BF0B9EC48F0000E63ECD8
:103F00002BF0DAEF1FF06BEC41F049EC43F0FF0EC1
:103F100063EC2BF0B9EC48F0000E63EC2BF0DAEF19
:103F20001FF083EC41F049EC43F0FF0E63EC2BF003
:103F3000DAEF1FF0A0EC41F049EC43F0FF0E63EC28
:103F40002BF0B9EC48F0000E63EC2BF0DAEF1FF029
:103F5000B8EC41F049EC43F0FF0E63EC2BF0B9EC08
:103F600048F0000E63EC2BF0B9EC48F0000E63EC67
:103F70002BF0DAEF1FF0CBEC41F049EC43F0FF0EF1
:103F800063EC2BF0B9EC48F0000E63EC2BF0DAEFA9
:103F90001FF0E3EC41F049EC43F0FF0E63EC2BF033
:103FA000B9EC48F0000E63EC2BF0B9EC48F0000ED1
:103FB00063EC2BF03FB6E1EF1FF03F861A504A6EDC
:103FC0004B6E94EC32F028EC2BF0400E31EC2BF0E1
:103FD000BD0E4AEC2BF0405040EC3AF089EC3AF040
:103FE0003F82FEEF20F0B9EC45F0000E63EC2BF0C1
:103FF000C9EC45F0000E63EC2BF0D9EC45F0000E57
:1040000063EC2BF089EC45F0000E63EC2BF0B9EC7F
:1040100046F0000E63EC2BF029EC46F0000E63EC4A
:104020002BF0A9EC46F0000E63EC2BF0B9EC48F055
:1040300029EC46F0000E63EC2BF059EC46F028EC2E
:104040002BF0400E31EC2BF0B90E4AEC2BF0000EA9
:1040500063EC2BF089EC45F0000E63EC2BF0B9EC2F
:1040600045F0000E63EC2BF025EC2BF0670E31ECE5
:104070002BF0BC0E4AEC2BF03FB053EF20F0000EBB
:1040800063EC2BF0F9EC46F0000E63EC2BF0C9EC7E
:1040900045F0000E63EC2BF099EC46F0000E63EC5B
:1040A0002BF065EF20F0FF0E63EC2BF099EC48F05D
:1040B000FF0E63EC2BF059EC47F0FF0E63EC2BF096
:1040C00039EC48F0FF0E63EC2BF028EC2BF0440E9B
:1040D00031EC2BF0BC0E4AEC2BF03FB084EF20F01B
:1040E000FF0E63EC2BF0E9EC47F0FF0E63EC2BF0D6
:1040F000C9EC48F0FF0E63EC2BF0F9EC47F0FF0E33
:1041000063EC2BF096EF20F0000E63EC2BF049EC03
:1041100046F0000E63EC2BF0B9EC48F0000E63ECB7
:104120002BF059EC46F0000E63EC2BF080B0AFEFB3
:1041300020F0070E555CD8B4A1EF20F0552AB1EF5E
:1041400020F0556A3EB0B1EF20F03FB0ABEF20F069
:104150003F80ACEF20F03F903E80B1EF20F03E90EA
:10416000556A84B6CAEF20F0070E545CD8B4BCEF91
:1041700020F0542ACCEF20F0546A3EBCCCEF20F063
:104180003FB0C6EF20F03F80C7EF20F03F903E8C5D
:10419000CCEF20F03E9C546A80B8FCEF20F0070E74
:1041A000575CD8B4D7EF20F0572AFEEF20F0576ABB
:1041B0003EB8FEEF20F0436A466A4DEC2CF03FA07B
:1041C000F8EF20F0080E116E040E126E4B0E136EF7
:1041D000BB0E146E9B0E156E880E166E7F0E176E3C
:1041E0007F0E186E000E196E000E1A6E6AEC2CF01F
:1041F0003F903E8823EF01F03E98576A80BA1AEF4D
:1042000021F0070E565CD8B409EF21F0562A1CEFB6
:1042100021F0566A3EBA23EF01F0000E436E3E8A4B
:10422000466A4DEC2CF03F903F923F96496A4A6AAD
:1042300023EF01F03E9A566A23EF01F025EC2BF0B4
:10424000410E31EC2BF0B80E4AEC2BF0700E63EC03
:104250002BF0100E63EC2BF0100E63EC2BF0100E15
:1042600063EC2BF0000E63EC2BF0C9EC45F0000E74
:1042700063EC2BF0C9EC45F0000E63EC2BF069EC1D
:1042800046F0000E63EC2BF089EC46F0000E63EC78
:104290002BF059EC46F0000E63EC2BF039EC46F0B5
:1042A000000E63EC2BF0B9EC48F0D9EC46F0000EB0
:1042B00063EC2BF089EC46F0000E63EC2BF009EC7C
:1042C00046F028EC2BF0400E31EC2BF0B80E4AEC07
:1042D0002BF0000E63EC2BF0A9EC46F0000E63EC23
:1042E0002BF0C9EC45F0000E63EC2BF0082A320EDF
:1042F000085CD8B481EF21F0100E63EC2BF076EF60
:1043000021F0086A700E63EC2BF0000E445CD8B408
:1043100091EF21F0010E445CD8B439EF25F023EF82
:1043200001F025EC2BF0460E31EC2BF0B90E4AECE7
:104330002BF099EC46F0000E63EC2BF0C9EC45F045
:10434000000E63EC2BF029EC46F0000E63EC2BF032
:10435000C9EC45F0000E63EC2BF0A9EC45F0000E23
:1043600063EC2BF0A9EC46F0000E63EC2BF0B9ECFB
:1043700048F089EC45F0000E63EC2BF0B9EC45F009
:10438000000E63EC2BF0B9EC45F028EC2BF0400E5E
:1043900031EC2BF0B90E4AEC2BF0000E63EC2BF055
:1043A00089EC46F0000E63EC2BF0C9EC45F0000EF2
:1043B00063EC2BF099EC46F0000E63EC2BF099ECDB
:1043C00046F0000E63EC2BF080B0FFEF21F0070EFB
:1043D000555CD8B4EFEF21F0552A01EF22F0556A71
:1043E0003EB001EF22F00B0E475CD8B4FBEF21F09A
:1043F000472AFCEF21F0476A3E8001EF22F03E9011
:10440000556A84B61DEF22F0070E545CD8B40CEF49
:1044100022F0542A1FEF22F0546A3EBC1FEF22F014
:10442000000E475CD8B418EF22F047061AEF22F0CE
:104430000B0E476E3E8C1FEF22F03E9C546A25EC1B
:104440002BF04A0E31EC2BF0BB0E4AEC2BF0000E99
:10445000475CD8B440EF22F0000E63EC2BF0A9ECDF
:1044600042F0000E63EC2BF0A9EC42F0000E63EC7E
:104470002BF0F9EC45F0000E63EC2BF052EF22F03C
:10448000FF0E63EC2BF049EC43F0FF0E63EC2BF0D6
:1044900049EC43F0FF0E63EC2BF089EC47F0FF0E84
:1044A00063EC2BF025EC2BF0670E31EC2BF0BB0E00
:1044B0004AEC2BF0010E475CD8B473EF22F0000EEB
:1044C00063EC2BF0A9EC42F0000E63EC2BF0B9EC9E
:1044D00042F0000E63EC2BF0F9EC45F0000E63ECBB
:1044E0002BF085EF22F0FF0E63EC2BF049EC43F04C
:1044F000FF0E63EC2BF059EC43F0FF0E63EC2BF056
:1045000089EC47F0FF0E63EC2BF028EC2BF0440E07
:1045100031EC2BF0BB0E4AEC2BF0020E475CD8B40A
:10452000A6EF22F0000E63EC2BF0A9EC42F0000E97
:1045300063EC2BF0C9EC42F0000E63EC2BF0F9ECCD
:1045400045F0000E63EC2BF0B8EF22F0FF0E63ECA9
:104550002BF049EC43F0FF0E63EC2BF069EC43F0D9
:10456000FF0E63EC2BF089EC47F0FF0E63EC2BF0B1
:1045700028EC2BF0610E31EC2BF0BB0E4AEC2BF04B
:10458000030E475CD8B4D9EF22F0000E63EC2BF099
:10459000A9EC42F0000E63EC2BF0D9EC42F0000ED7
:1045A00063EC2BF0F9EC45F0000E63EC2BF0EBEF35
:1045B00022F0FF0E63EC2BF049EC43F0FF0E63ECAE
:1045C0002BF079EC43F0FF0E63EC2BF089EC47F015
:1045D000FF0E63EC2BF025EC2BF04A0E31EC2BF0A8
:1045E000BC0E4AEC2BF0040E475CD8B40CEF23F061
:1045F000000E63EC2BF0A9EC42F0000E63EC2BF004
:10460000E9EC42F0000E63EC2BF0F9EC45F0000E03
:1046100063EC2BF01EEF23F0FF0E63EC2BF049EC64
:1046200043F0FF0E63EC2BF089EC43F0FF0E63ECDC
:104630002BF089EC47F0FF0E63EC2BF025EC2BF010
:10464000670E31EC2BF0BC0E4AEC2BF0050E475CEC
:10465000D8B43FEF23F0000E63EC2BF0A9EC42F04E
:10466000000E63EC2BF0F9EC42F0000E63EC2BF043
:10467000F9EC45F0000E63EC2BF051EF23F0FF0E48
:1046800063EC2BF049EC43F0FF0E63EC2BF099EC5C
:1046900043F0FF0E63EC2BF089EC47F0FF0E63EC68
:1046A0002BF028EC2BF0440E31EC2BF0BC0E4AEC36
:1046B0002BF0060E475CD8B472EF23F0000E63ECCB
:1046C0002BF0A9EC42F0000E63EC2BF009EC43F068
:1046D000000E63EC2BF0F9EC45F0000E63EC2BF0D0
:1046E00084EF23F0FF0E63EC2BF049EC43F0FF0E58
:1046F00063EC2BF0A9EC43F0FF0E63EC2BF089EC9C
:1047000047F0FF0E63EC2BF028EC2BF0610E31EC40
:104710002BF0B40E4AEC2BF0070E475CD8B4A5EF93
:1047200023F0000E63EC2BF0A9EC42F0000E63ECDA
:104730002BF019EC43F0000E63EC2BF0F9EC45F094
:10474000000E63EC2BF0B7EF23F0FF0E63EC2BF0C1
:1047500049EC43F0FF0E63EC2BF0B9EC43F0FF0E95
:1047600063EC2BF089EC47F0FF0E63EC2BF025ECAB
:104770002BF04A0E31EC2BF0BD0E4AEC2BF0080E5C
:10478000475CD8B4D8EF23F0000E63EC2BF0A9EC13
:1047900042F0000E63EC2BF029EC43F0000E63ECCA
:1047A0002BF0F9EC45F0000E63EC2BF0EAEF23F070
:1047B000FF0E63EC2BF049EC43F0FF0E63EC2BF0A3
:1047C000C9EC43F0FF0E63EC2BF089EC47F0FF0ED1
:1047D00063EC2BF025EC2BF0670E31EC2BF0BD0ECB
:1047E0004AEC2BF0090E475CD8B40BEF24F0000E16
:1047F00063EC2BF0A9EC42F0000E63EC2BF039ECEB
:1048000043F0000E63EC2BF0F9EC45F0000E63EC86
:104810002BF01DEF24F0FF0E63EC2BF049EC43F07E
:10482000FF0E63EC2BF0D9EC43F0FF0E63EC2BF0A2
:1048300089EC47F0FF0E63EC2BF025EC2BF04A0ED1
:1048400031EC2BF0BE0E4AEC2BF00A0E475CD8B4CC
:1048500059EF24F0000E63EC2BF059EC46F0000EFB
:1048600063EC2BF0A9EC46F0000E63EC2BF0F9ECB6
:1048700045F0000E63EC2BF0C9EC45F0000E63EC44
:104880002BF089EC46F0000E63EC2BF0B9EC48F00D
:1048900099EC46F0000E63EC2BF0C9EC45F0000EED
:1048A00063EC2BF0A9EC46F0000E63EC2BF086EFE6
:1048B00024F0FF0E63EC2BF0F9EC47F0FF0E63ECF5
:1048C0002BF049EC48F0FF0E63EC2BF089EC47F03D
:1048D000FF0E63EC2BF059EC47F0FF0E63EC2BF06E
:1048E00029EC48F0FF0E63EC2BF0C9EC48F039ECF2
:1048F00048F0FF0E63EC2BF059EC47F0FF0E63EC31
:104900002BF049EC48F0FF0E63EC2BF025EC2BF07C
:104910004A0E31EC2BF0BF0E4AEC2BF00B0E475C2D
:10492000D8B4D9EF24F0000E63EC2BF089EC45F0FD
:10493000000E63EC2BF029EC46F0000E63EC2BF03C
:1049400029EC46F0000E63EC2BF0B9EC48F089EC52
:1049500046F0000E63EC2BF0C9EC45F0000E63EC62
:104960002BF0E9EC45F0000E63EC2BF009EC46F07F
:10497000000E63EC2BF099EC46F0000E63EC2BF08C
:1049800028EC2BF0400E31EC2BF0BF0E4AEC2BF054
:10499000A9EC46F0000E63EC2BF0C9EC45F0000EDC
:1049A00063EC2BF089EC46F0000E63EC2BF01DEF6E
:1049B00025F0FF0E63EC2BF019EC47F0FF0E63ECD3
:1049C0002BF0C9EC47F0FF0E63EC2BF0C9EC47F07D
:1049D000FF0E63EC2BF0C9EC48F029EC48F0FF0E19
:1049E00063EC2BF059EC47F0FF0E63EC2BF079EC05
:1049F00047F0FF0E63EC2BF099EC47F0FF0E63ECF1
:104A00002BF039EC48F0FF0E63EC2BF028EC2BF088
:104A1000400E31EC2BF0BF0E4AEC2BF049EC48F085
:104A2000FF0E63EC2BF059EC47F0FF0E63EC2BF01C
:104A300029EC48F0FF0E63EC2BF0E6EC2EF080B88A
:104A400035EF25F0070E575CD8B42AEF25F0572A2A
:104A500037EF25F0576A3EB837EF25F0010E446E68
:104A60004DEC2CF03E8837EF25F03E98576A23EF47
:104A700001F025EC2BF0460E31EC2BF0B90E4AEC90
:104A80002BF0000E475CD8B47AEF25F0010E475C9E
:104A9000D8B482EF25F0020E475CD8B48AEF25F037
:104AA000030E475CD8B492EF25F0040E475CD8B4EF
:104AB0009AEF25F0050E475CD8B4A2EF25F0060E5C
:104AC000475CD8B4AAEF25F0070E475CD8B4B2EF24
:104AD00025F0080E475CD8B4BAEF25F0090E475C04
:104AE000D8B4C2EF25F00A0E475CD8B4CAEF25F05F
:104AF00024EF26F0F6EC3CF027EC35F0C0EC35F076
:104B0000B5EF26F04FEC3DF027EC35F0C0EC35F07A
:104B1000B5EF26F0A8EC3DF027EC35F0C0EC35F011
:104B2000B5EF26F001EC3EF027EC35F0C0EC35F0A7
:104B3000B5EF26F05AEC3EF027EC35F0C0EC35F03E
:104B4000B5EF26F0B3EC3EF027EC35F0C0EC35F0D5
:104B5000B5EF26F05CEC3FF027EC35F0C0EC35F01B
:104B6000B5EF26F0EAEC3FF027EC35F0C0EC35F07D
:104B7000B5EF26F059EC40F027EC35F0C0EC35F0FD
:104B8000B5EF26F0E2EC40F027EC35F0C0EC35F064
:104B9000B5EF26F0000E63EC2BF059EC46F0000E5A
:104BA00063EC2BF0A9EC46F0000E63EC2BF0F9EC73
:104BB00045F0000E63EC2BF0C9EC45F0000E63EC01
:104BC0002BF089EC46F0000E63EC2BF0B9EC48F0CA
:104BD00099EC46F0000E63EC2BF0C9EC45F0000EAA
:104BE00063EC2BF0A9EC46F0000E63EC2BF028EC04
:104BF0002BF0400E31EC2BF0B90E4AEC2BF0000EEE
:104C000063EC2BF0000E63EC2BF0D9EC46F0000EB9
:104C100063EC2BF089EC46F0000E63EC2BF009EC12
:104C200046F0000E63EC2BF0A9EC46F0000E63ECAE
:104C30002BF0C9EC45F0000E63EC2BF027EC35F0BF
:104C4000C0EC35F0B5EF26F089EC45F0000E63ECD2
:104C50002BF029EC46F0000E63EC2BF029EC46F02B
:104C6000000E63EC2BF0B9EC48F089EC46F0000E36
:104C700063EC2BF0C9EC45F0000E63EC2BF0E9EC93
:104C800045F0000E63EC2BF009EC46F0000E63ECEF
:104C90002BF099EC46F0000E63EC2BF0A9EC46F0FB
:104CA00028EC2BF0400E31EC2BF0B90E4AEC2BF037
:104CB000000E63EC2BF0C9EC45F0000E63EC2BF01A
:104CC00089EC46F0000E63EC2BF0B9EC48F0D9EC1F
:104CD00046F0000E63EC2BF089EC46F0000E63EC1E
:104CE0002BF009EC46F0000E63EC2BF0A9EC46F03B
:104CF000000E63EC2BF0C9EC45F0000E63EC2BF0DA
:104D000027EC35F080B8B3EF26F0070E575CD8B427
:104D10008DEF26F0572AB5EF26F0576A3EB8B5EF6B
:104D200026F03FACACEF26F04DEC2CF0F1EC48F067
:104D300004EC49F017EC49F02AEC49F03DEC49F05D
:104D400050EC49F063EC49F076EC49F089EC49F01D
:104D50009CEC49F0AFEC49F0446A476A3F9C3F90B5
:104D60003E8823EF01F03E98576A80BA23EF01F0A6
:104D7000070E565CD8B4C0EF26F0562A23EF01F098
:104D8000566A000E446E3E8A476A4DEC2CF03F9CFA
:104D900023EF01F025EC2BF0410E31EC2BF0B80E97
:104DA0004AEC2BF0700E63EC2BF0100E63EC2BF042
:104DB000100E63EC2BF0100E63EC2BF0000E63EC86
:104DC0002BF059EC46F0000E63EC2BF0A9EC46F00A
:104DD000000E63EC2BF0F9EC45F0000E63EC2BF0C9
:104DE000C9EC45F0000E63EC2BF089EC46F0000EA8
:104DF00063EC2BF0B9EC48F099EC46F0000E63EC54
:104E00002BF0C9EC45F0000E63EC2BF0A9EC46F05A
:104E1000000E63EC2BF0A9EC46F028EC2BF0400ED2
:104E200031EC2BF0B80E4AEC2BF0000E63EC2BF0BB
:104E300009EC46F0000E63EC2BF049EC46F0000E56
:104E400063EC2BF0E9EC45F0000E63EC2BF0082A44
:104E50002C0E085CD8B432EF27F0100E63EC2BF068
:104E600027EF27F0086A700E63EC2BF025EC2BF08F
:104E7000460E31EC2BF0BF0E4AEC2BF099EC46F0CD
:104E8000000E63EC2BF059EC46F0000E63EC2BF0B7
:104E9000D9EC45F0000E63EC2BF0A9EC46F0000EC7
:104EA00063EC2BF0D9EC46F0000E63EC2BF089ECB0
:104EB00045F0000E63EC2BF089EC46F0000E63EC3D
:104EC0002BF0C9EC45F0000E63EC2BF0B9EC48F088
:104ED000C9EC46F028EC2BF0400E31EC2BF0BF0E65
:104EE0004AEC2BF0000E63EC2BF0C9EC45F0000E01
:104EF00063EC2BF089EC46F0000E63EC2BF099ECA0
:104F000046F0000E63EC2BF009EC46F0000E63EC6B
:104F10002BF059EC46F0000E63EC2BF049EC46F018
:104F2000000E63EC2BF0B9EC48F0000E63EC2BF0B4
:104F3000B9EC42F0000E63EC2BF0000E63EC2BF0AA
:104F4000400E63EC2BF0000E63EC2BF0A9EC42F06A
:104F5000000E63EC2BF0B9EC42F0000E63EC2BF08A
:104F600025EC2BF0450E31EC2BF0BA0E4AEC2BF071
:104F70004CBEFCEF27F0000E485CD8A4FCEF27F0F5
:104F8000FF0E63EC2BF059EC47F0FF0E63EC2BF0B7
:104F900029EC48F0FF0E63EC2BF029EC48F0FF0EF3
:104FA00063EC2BF0F9EC47F0FF0E63EC2BF029ECEF
:104FB00048F0FF0E63EC2BF0C9EC48F089EC47F0A9
:104FC000FF0E63EC2BF0F9EC47F0FF0E63EC2BF0D7
:104FD000C9EC47F0FF0E63EC2BF049EC47F028ECEE
:104FE0002BF0400E31EC2BF0BA0E4AEC2BF0FF0EFA
:104FF00063EC2BF036EF28F0000E63EC2BF0C9ECDD
:1050000045F0000E63EC2BF089EC46F0000E63ECEB
:105010002BF089EC46F0000E63EC2BF059EC46F0D7
:10502000000E63EC2BF089EC46F0000E63EC2BF0E5
:10503000B9EC48F0F9EC45F0000E63EC2BF059ECBC
:1050400046F0000E63EC2BF029EC46F0000E63EC0A
:105050002BF0B9EC45F028EC2BF0400E31EC2BF0A6
:10506000BA0E4AEC2BF0000E63EC2BF025EC2BF083
:10507000450E31EC2BF0BB0E4AEC2BF04CBE75EF1D
:1050800028F0010E485CD8A475EF28F0FF0E63EC01
:105090002BF049EC48F0FF0E63EC2BF089EC48F064
:1050A000FF0E63EC2BF0C9EC48F0F9EC47F0FF0E73
:1050B00063EC2BF059EC48F0FF0E63EC2BF049EC5D
:1050C00048F0FF0E63EC2BF009EC48F0FF0E63ECA8
:1050D0002BF059EC48F0FF0E63EC2BF049EC48F054
:1050E000FF0E63EC2BF0A2EF28F0000E63EC2BF028
:1050F000A9EC46F0000E63EC2BF0E9EC46F0000E54
:1051000063EC2BF0B9EC48F059EC46F0000E63EC80
:105110002BF0B9EC46F0000E63EC2BF0A9EC46F056
:10512000000E63EC2BF069EC46F0000E63EC2BF004
:10513000B9EC46F0000E63EC2BF0A9EC46F0000E43
:1051400063EC2BF025EC2BF0450E31EC2BF0BC0E74
:105150004AEC2BF04CBEEEEF28F0020E485CD8A4CF
:10516000EEEF28F0FF0E63EC2BF039EC48F0FF0E69
:1051700063EC2BF059EC47F0FF0E63EC2BF0C9EC1D
:1051800047F0FF0E63EC2BF059EC47F0FF0E63EC99
:105190002BF039EC47F0FF0E63EC2BF049EC48F0B4
:1051A000FF0E63EC2BF0C9EC48F059EC48F0FF0E11
:1051B00063EC2BF039EC48F0FF0E63EC2BF029EC9C
:1051C00047F028EC2BF0400E31EC2BF0BC0E4AECF3
:1051D0002BF0FF0E63EC2BF028EF29F0000E63ECB0
:1051E0002BF099EC46F0000E63EC2BF0C9EC45F087
:1051F000000E63EC2BF029EC46F0000E63EC2BF074
:10520000C9EC45F0000E63EC2BF0A9EC45F0000E64
:1052100063EC2BF0A9EC46F0000E63EC2BF0B9EC3C
:1052200048F0B9EC46F0000E63EC2BF099EC46F038
:10523000000E63EC2BF099EC45F028EC2BF0400EBF
:1052400031EC2BF0BC0E4AEC2BF0000E63EC2BF093
:105250004CBE66EF29F080B046EF29F0070E555C92
:10526000D8B436EF29F0552A48EF29F0556A3EB0F8
:1052700048EF29F0020E485CD8B442EF29F0482AE2
:1052800043EF29F0486A3E8048EF29F03E90556A86
:1052900084B664EF29F0070E545CD8B453EF29F0BC
:1052A000542A66EF29F0546A3EBC66EF29F0000EDE
:1052B000485CD8B45FEF29F0480661EF29F0020E90
:1052C000486E3E8C66EF29F03E9C546A4CBE80EFDF
:1052D00029F080B87EEF29F0070E575CD8B474EF40
:1052E00029F0572A80EF29F0576A3EB880EF29F05D
:1052F0004C8E4C504D6E3E8880EF29F03E98576A98
:105300004CAE9AEF29F080BA98EF29F0070E565C60
:10531000D8B48EEF29F0562A9AEF29F0566A3EBA91
:105320009AEF29F04C9E4DEC2CF03E8A9AEF29F032
:105330003E9A566A4CAEB6EF29F080B8B4EF29F029
:10534000070E575CD8B4A8EF29F0572AB6EF29F01A
:10535000576A3EB8B6EF29F04D504C6E4C9E4DEC5E
:105360002CF03E88B6EF29F03E98576A4CAE11EF0C
:105370002AF080B0E3EF29F0070E555CD8B4C4EFF3
:1053800029F0552AE5EF29F0556A3EB0E5EF29F0FE
:10539000000E485CD8B4D9EF29F0010E485CD8B4AF
:1053A000DCEF29F0020E485CD8B4DFEF29F0E0EF23
:1053B00029F04D70E0EF29F04D72E0EF29F04D74C7
:1053C0003E80E5EF29F03E90556A84B60FEF2AF053
:1053D000070E545CD8B4F0EF29F0542A11EF2AF0EC
:1053E000546A3EBC11EF2AF0000E485CD8B405EFB9
:1053F0002AF0010E485CD8B408EF2AF0020E485C8F
:10540000D8B40BEF2AF00CEF2AF04D700CEF2AF015
:105410004D720CEF2AF04D743E8C11EF2AF03E9C39
:10542000546A4CAE20EF2BF0000E485CD8B425EF48
:105430002AF0010E485CD8B462EF2AF0020E485CF4
:10544000D8B4D1EF2AF020EF2BF028EC2BF0460E49
:1054500031EC2BF0BA0E4AEC2BF04DA049EF2AF0BC
:10546000FF0E63EC2BF089EC47F0FF0E63EC2BF0A2
:10547000F9EC47F0FF0E63EC2BF0C9EC47F0FF0EA0
:1054800063EC2BF049EC47F0FF0E63EC2BF020EFC0
:105490002BF0FF0E63EC2BF069EC47F0FF0E63EC92
:1054A0002BF029EC48F0FF0E63EC2BF059EC47F0A1
:1054B000FF0E63EC2BF059EC47F0FF0E63EC2BF082
:1054C00020EF2BF028EC2BF0460E31EC2BF0BB0E2E
:1054D0004AEC2BF04DA29FEF2AF0FF0E63EC2BF06D
:1054E00099EC47F0FF0E63EC2BF0E9EC47F0FF0E70
:1054F00063EC2BF049EC48F0FF0E63EC2BF059EC19
:1055000047F0FF0E63EC2BF029EC48F0FF0E63EC44
:105510002BF0C9EC47F0FF0E63EC2BF0F9EC47F0F1
:10552000FF0E63EC2BF039EC47F0FF0E63EC2BF031
:10553000B9EC47F0FF0E63EC2BF020EF2BF0FF0EE1
:1055400063EC2BF069EC47F0FF0E63EC2BF029ECD9
:1055500048F0FF0E63EC2BF059EC47F0FF0E63ECC4
:105560002BF059EC47F0FF0E63EC2BF0B9EC48F050
:10557000000E63EC2BF0B9EC48F0000E63EC2BF05E
:10558000B9EC48F0000E63EC2BF0B9EC48F0000EDB
:1055900063EC2BF0B9EC48F0000E63EC2BF020EF3D
:1055A0002BF028EC2BF0460E31EC2BF0BC0E4AEC25
:1055B0002BF04DA4FFEF2AF0FF0E63EC2BF019EC5B
:1055C00047F0FF0E63EC2BF059EC48F0FF0E63EC54
:1055D0002BF049EC48F0FF0E63EC2BF0F9EC47F0B0
:1055E000FF0E63EC2BF0B9EC48F0000E63EC2BF0EF
:1055F000B9EC48F0000E63EC2BF020EF2BF0FF0E1F
:1056000063EC2BF0D9EC47F0FF0E63EC2BF019ECB8
:1056100047F0FF0E63EC2BF0E9EC47F0FF0E63EC74
:105620002BF059EC48F0FF0E63EC2BF019EC47F02F
:10563000FF0E63EC2BF0C9EC47F0FF0E63EC2BF090
:105640004CAEE6EC2EF023EF01F08C888B9E12001E
:105650008C988B8E12008C888B8E12008C988B9E6F
:105660001200016E2AEC2CF001508A6E8C9C8C9EEC
:10567000000000008C8A0000000000000000000014
:105680000000000000008C9A0000000000000000F4
:1056900000001200026E2AEC2CF002508A6E8C9CE4
:1056A0008C9E000000008C8A0000000000000000BA
:1056B00000000000000000008C9A000000000000C4
:1056C000000000001200006E2AEC2CF03FBE7FECC0
:1056D0002BF000508A6E8C9C8C8E000000008C8A0F
:1056E00000000000000000000000000000000000BA
:1056F0008C9A000000000000000000001200000E64
:10570000515CD8B4A4EF2BF0010E515CD8B4BDEFBE
:105710002BF0020E515CD8B4D4EF2BF0030E515C89
:10572000D8B4E9EF2BF0040E515CD8B4FCEF2BF0A9
:10573000050E515CD8B40DEF2CF0060E515CD8B4B8
:105740001CEF2CF029EF2CF050B0B2EF2BF0004200
:10575000004200420042004200420042010E001698
:1057600029EF2CF000460046004600460046004661
:105770000046800E001629EF2CF050B0CAEF2BF037
:10578000004200420042004200420042030E001666
:1057900029EF2CF000460046004600460046004631
:1057A000C00E001629EF2CF050B0E0EF2BF00042B5
:1057B0000042004200420042070E001629EF2CF082
:1057C00000460046004600460046E00E001629EF5F
:1057D0002CF050B0F4EF2BF00042004200420042A7
:1057E0000F0E001629EF2CF000460046004600463A
:1057F000F00E001629EF2CF050B006EF2CF000420E
:10580000004200421F0E001629EF2CF00046004611
:105810000046F80E001629EF2CF050B016EF2CF0D1
:10582000004200423F0E001629EF2CF000460046D1
:10583000FC0E001629EF2CF050B024EF2CF00042A3
:105840007F0E001629EF2CF00046FE0E001629EF01
:105850002CF012000F01FF0E936E00018C8C8C9EB9
:10586000000000008C8A0000000000000000000022
:105870000000000000008C9A000000000000000002
:10588000000000000000000081BE32EF2CF08C9C74
:105890000F01000E936E000112002BEC2BF0400E56
:1058A00031EC2BF0B80E4AEC2BF0000E63EC2BF031
:1058B000012A800E015CD8A455EF2CF0022A4BEC93
:1058C0002BF0400E31EC2BF0C00E025CD8A455EF4B
:1058D0002CF012008B8000008B9272EC37F08B82E0
:1058E00072EC37F087EC2CF09DEC2CF0B2EC2CF045
:1058F000C7EC2CF0DCEC2CF0F1EC2CF006EC2DF0ED
:105900001BEC2DF030EC2DF045EC2DF012008B90BF
:1059100000005AEC2DF08B9400008B8600008B96D3
:105920000000000E386E85EC2DF011503C6E9AECA4
:105930002DF08B948B968B8012008B905AEC2DF06F
:105940008B9400008B8600008B960000010E386E51
:1059500085EC2DF012503C6E9AEC2DF08B948B96CA
:105960008B8012008B905AEC2DF08B9400008B866C
:1059700000008B960000020E386E85EC2DF013505F
:105980003C6E9AEC2DF08B948B968B8012008B9052
:105990005AEC2DF08B9400008B8600008B96000053
:1059A000030E386E85EC2DF014503C6E9AEC2DF001
:1059B0008B948B968B8012008B905AEC2DF08B94ED
:1059C00000008B8600008B960000040E386E85EC7C
:1059D0002DF015503C6E9AEC2DF08B948B968B80AD
:1059E00012008B905AEC2DF08B9400008B860000F7
:1059F0008B960000050E386E85EC2DF016503C6E2F
:105A00009AEC2DF08B948B968B8012008B905AEC35
:105A10002DF08B9400008B8600008B960000060E04
:105A2000386E85EC2DF017503C6E9AEC2DF08B946F
:105A30008B968B8012008B905AEC2DF08B9400008B
:105A40008B8600008B960000070E386E85EC2DF0DB
:105A500018503C6E9AEC2DF08B948B968B80120034
:105A60008B905AEC2DF08B9400008B8600008B9667
:105A70000000080E386E85EC2DF019503C6E9AEC43
:105A80002DF08B948B968B8012008B905AEC2DF01E
:105A90008B9400008B8600008B960000090E386EF8
:105AA00085EC2DF01A503C6E9AEC2DF08B948B9671
:105AB0008B8012008B9400008B8600008B96000078
:105AC0008B9400008B8600008B9600008B84000076
:105AD0008B8600008B9600008B9400008B86000064
:105AE0008B9600008B9400008B8600008B96000044
:105AF0008B9400008B8600008B9600008B94000036
:105B00008B8600008B960000120038BE8BEF2DF0C4
:105B10008B948DEF2DF08B8400008B8600008B968C
:105B20000000392A3846080E395CD8A485EF2DF0DC
:105B3000396A12003CBEA0EF2DF08B94A2EF2DF03D
:105B40008B8400008B8600008B9600003A2A3C462E
:105B5000080E3A5CD8A49AEF2DF03A6A12008B90A6
:105B60005AEC2DF08B9400008B8600008B96000081
:105B70000A0E386E85EC2DF08B80000000000000CE
:105B80008B905AEC2DF08B8400008B8600008B9656
:105B90000000000000000000D2EC2DF08B948B96EA
:105BA0008B8012008B8683A0D9EF2DF03B80DAEF3B
:105BB0002DF03B903A2A8B96080E3A5CD8B4E4EF6D
:105BC0002DF03B46D2EF2DF03A6A3D2A010E3D5CA6
:105BD000D8A4EFEF2DF03B501B6ED2EF2DF0020E4C
:105BE0003D5CD8A4F8EF2DF03B501C6ED2EF2DF0A9
:105BF000030E3D5CD8A401EF2EF03B501D6ED2EF9A
:105C00002DF0040E3D5CD8A40AEF2EF03B501E6E22
:105C1000D2EF2DF0050E3D5CD8A413EF2EF03B50D3
:105C20001F6ED2EF2DF0060E3D5CD8A41CEF2EF0B7
:105C30003B50206ED2EF2DF0070E3D5CD8A425EF2F
:105C40002EF03B50216ED2EF2DF0080E3D5CD8A413
:105C50002EEF2EF03B50226ED2EF2DF0090E3D5C60
:105C6000D8A437EF2EF03B50236ED2EF2DF00A0E62
:105C70003D5CD8A440EF2EF03B50246ED2EF2DF0C7
:105C80000B0E3D5CD8A449EF2EF03B50256ED2EFB1
:105C90002DF00C0E3D5CD8A452EF2EF03B50266E3A
:105CA000D2EF2DF00D0E3D5CD8A45BEF2EF03B50F3
:105CB000276ED2EF2DF00E0E3D5CD8A464EF2EF0CF
:105CC0003B50286ED2EF2DF00F0E3D5CD8A46DEF47
:105CD0002EF03B50296ED2EF2DF0100E3D5CD8A473
:105CE00076EF2EF03B502A6ED2EF2DF0110E3D5C78
:105CF000D8A47FEF2EF03B502B6ED2EF2DF0120E7A
:105D00003D5CD8A488EF2EF03B502C6ED2EF2DF0E6
:105D1000130E3D5CD8A491EF2EF03B502D6ED2EFC8
:105D20002DF0140E3D5CD8A49AEF2EF03B502E6E51
:105D3000D2EF2DF0150E3D5CD8A4A3EF2EF03B5012
:105D40002F6ED2EF2DF0160E3D5CD8A4ACEF2EF0E6
:105D50003B50306ED2EF2DF0170E3D5CD8A4B5EF5E
:105D60002EF03B50316ED2EF2DF0180E3D5CD8A4D2
:105D7000BEEF2EF03B50326ED2EF2DF0190E3D5C8F
:105D8000D8A4C7EF2EF03B50336ED2EF2DF01A0E91
:105D90003D5CD8A4D0EF2EF03B50346ED2EF2DF006
:105DA0001B0E3D5CD8A4D9EF2EF03B50356ED2EFE0
:105DB0002DF01C0E3D5CD8A4E2EF2EF03B50366E69
:105DC000D2EF2DF03B50376E3D6A120080BAFCEFE7
:105DD0002EF0070E565CD8B4F1EF2EF0562AFEEFE7
:105DE0002EF0566A3EBA12004DEC2CF0416A466A1B
:105DF000476A486A3E8A12003E9A566A1200000EAE
:105E0000405CD8A428EF2FF0E9EC45F0000E63ECDD
:105E10002BF049EC46F0000E63EC2BF0B9EC45F0AA
:105E2000000E63EC2BF0B9EC48F0000E63EC2BF0A5
:105E3000B9EC48F0000E63EC2BF0B9EC48F0000E22
:105E400063EC2BF0B9EC48F0000E63EC2BF0120081
:105E5000010E405CD8A451EF2FF0C9EC45F0000EC4
:105E600063EC2BF039EC46F0000E63EC2BF069ECA0
:105E700046F0000E63EC2BF0F9EC45F0000E63ECFD
:105E80002BF0B9EC48F0000E63EC2BF0B9EC48F0C5
:105E9000000E63EC2BF0B9EC48F0000E63EC2BF035
:105EA0001200020E405CD8A47AEF2FF009EC46F005
:105EB000000E63EC2BF049EC46F0000E63EC2BF087
:105EC000A9EC46F0000E63EC2BF0B9EC48F0000EA4
:105ED00063EC2BF0B9EC48F0000E63EC2BF0B9EC5E
:105EE00048F0000E63EC2BF0B9EC48F0000E63ECC8
:105EF0002BF01200030E405CD8A4A3EF2FF0A9EC06
:105F000045F0000E63EC2BF0B9EC48F0000E63ECAA
:105F10002BF099EC46F0000E63EC2BF0A9EC46F068
:105F2000000E63EC2BF089EC45F0000E63EC2BF0D7
:105F3000B9EC48F0000E63EC2BF0B9EC48F0000E21
:105F400063EC2BF01200040E405CD8A4CCEF2FF0D1
:105F5000B9EC46F0000E63EC2BF0B9EC48F0000E03
:105F600063EC2BF0B9EC45F0000E63EC2BF089EC00
:105F700045F0000E63EC2BF0A9EC46F0000E63EC4C
:105F80002BF089EC45F0000E63EC2BF0B9EC48F0F7
:105F9000000E63EC2BF01200050E405CD8A4F5EF68
:105FA0002FF089EC46F0000E63EC2BF0B9EC48F0D2
:105FB000000E63EC2BF0C9EC45F0000E63EC2BF007
:105FC00089EC46F0000E63EC2BF089EC46F0000EF5
:105FD00063EC2BF0B9EC48F0000E63EC2BF0B9EC5D
:105FE00048F0000E63EC2BF01200060E405CD8A4C3
:105FF0001EEF30F049EC46F0000E63EC2BF0C9ECDC
:1060000046F0000E63EC2BF0B9EC48F0000E63ECA8
:106010002BF0C9EC45F0000E63EC2BF089EC46F058
:10602000000E63EC2BF089EC46F0000E63EC2BF0D5
:10603000B9EC48F0000E63EC2BF01200070E405C48
:10604000D8A447EF30F089EC46F0000E63EC2BF05B
:10605000A9EC45F0000E63EC2BF099EC45F0000E36
:1060600063EC2BF029EC46F0000E63EC2BF0B9EC5E
:1060700048F0000E63EC2BF0B9EC48F0000E63EC36
:106080002BF0B9EC48F0000E63EC2BF01200080E78
:10609000405CD8A470EF30F039EC43F0000E63ECB4
:1060A0002BF009EC43F0000E63EC2BF019EC46F0FA
:1060B000000E63EC2BF0F9EC45F0000E63EC2BF0D6
:1060C00009EC47F0000E63EC2BF0B9EC48F0000E41
:1060D00063EC2BF0B9EC48F0000E63EC2BF01200EF
:1060E000090E405CD8A499EF30F089EC45F0000E21
:1060F00063EC2BF0B9EC46F0000E63EC2BF0B9EC3E
:1061000045F0000E63EC2BF009EC46F0000E63EC5A
:106110002BF059EC46F0000E63EC2BF0B9EC48F094
:10612000000E63EC2BF0B9EC48F0000E63EC2BF0A2
:1061300012000A0E405CD8A4C2EF30F0C9EC46F061
:10614000000E63EC2BF029EC46F0000E63EC2BF014
:1061500089EC46F0000E63EC2BF0A9EC45F0000E44
:1061600063EC2BF019EC46F0000E63EC2BF0B9EC6D
:1061700048F0000E63EC2BF0B9EC48F0000E63EC35
:106180002BF012000B0E405CD8A4A4EF31F0A9EC68
:1061900046F0000E63EC2BF0E9EC46F0000E63ECE9
:1061A0002BF0B9EC48F0000E63EC2BF01550070B08
:1061B000406E000E405CD8A4F3EF30F089EC46F05E
:1061C000000E63EC2BF0E9EC46F0000E63EC2BF0D4
:1061D00069EC46F0000E63EC2BF0A9EC42F0000EE7
:1061E00063EC2BF01200010E405CD8A40DEF31F0EF
:1061F00089EC46F0000E63EC2BF0E9EC46F0000E63
:1062000063EC2BF069EC46F0000E63EC2BF0B9EC7C
:1062100042F0000E63EC2BF01200020E405CD8A49A
:1062200027EF31F089EC46F0000E63EC2BF0E9EC3F
:1062300046F0000E63EC2BF069EC46F0000E63ECC8
:106240002BF0C9EC42F0000E63EC2BF01200030EB1
:10625000405CD8A441EF31F0B9EC46F0000E63EC9D
:106260002BF099EC46F0000E63EC2BF099EC45F026
:10627000000E63EC2BF0B9EC48F0000E63EC2BF051
:106280001200040E405CD8A45BEF31F089EC46F0BC
:10629000000E63EC2BF0E9EC46F0000E63EC2BF003
:1062A00069EC46F0000E63EC2BF0E9EC42F0000ED6
:1062B00063EC2BF01200050E405CD8A475EF31F0B2
:1062C00089EC46F0000E63EC2BF0E9EC46F0000E92
:1062D00063EC2BF069EC46F0000E63EC2BF0F9EC6C
:1062E00042F0000E63EC2BF01200060E405CD8A4C6
:1062F0008FEF31F089EC46F0000E63EC2BF0E9EC07
:1063000046F0000E63EC2BF069EC46F0000E63ECF7
:106310002BF009EC43F0000E63EC2BF0120089EC3B
:1063200046F0000E63EC2BF0E9EC46F0000E63EC57
:106330002BF069EC46F0000E63EC2BF019EC43F007
:10634000000E63EC2BF012000C0E405CD8A4CDEFD5
:1063500031F0C9EC46F0000E63EC2BF0B9EC45F0DF
:10636000000E63EC2BF0B9EC45F0000E63EC2BF063
:10637000B9EC48F0000E63EC2BF0B9EC48F0000EDD
:1063800063EC2BF0B9EC48F0000E63EC2BF0B9ECA9
:1063900048F0000E63EC2BF012000D0E405CD8A408
:1063A000F6EF31F0F9EC45F0000E63EC2BF089ECE0
:1063B00046F0000E63EC2BF039EC46F0000E63EC77
:1063C0002BF0A9EC45F0000E63EC2BF019EC46F035
:1063D000000E63EC2BF0B9EC48F0000E63EC2BF0F0
:1063E000B9EC48F0000E63EC2BF0120089EC46F09B
:1063F000000E63EC2BF0C9EC45F0000E63EC2BF0C3
:1064000099EC46F0000E63EC2BF0C9EC45F0000E61
:1064100063EC2BF089EC46F0000E63EC2BF0C9EC3A
:1064200046F0000E63EC2BF0C9EC45F0000E63EC77
:106430002BF0120080B036EF32F0070E555CD8B466
:1064400025EF32F0552A38EF32F0556A3EB038EF7A
:1064500032F0000E495CD8A432EF32F0080E496EDB
:1064600033EF32F049063E8038EF32F03E90556A05
:1064700084B654EF32F0070E545CD8B443EF32F0D8
:10648000542A56EF32F0546A3EBC56EF32F0080EF2
:10649000495CD8A450EF32F0000E496E51EF32F053
:1064A000492A3E8C56EF32F03E9C546A120080B06E
:1064B00073EF32F0070E555CD8B462EF32F0552A14
:1064C00075EF32F0556A3EB075EF32F0010E495C5F
:1064D000D8A46FEF32F0080E496E70EF32F0490623
:1064E0003E8075EF32F03E90556A84B691EF32F0FF
:1064F000070E545CD8B480EF32F0542A93EF32F098
:10650000546A3EBC93EF32F0080E495CD8A48DEF7C
:1065100032F0010E496E8EEF32F0492A3E8C93EF35
:1065200032F03E9C546A1200080E495CD8B4AAEFBF
:1065300034F03FB4DAEF32F080B8AFEF32F0070E4C
:10654000575CD8B4A7EF32F0572AB1EF32F0576A50
:106550003EB86DEF33F03F843E88DAEF32F03E987C
:10656000576A25EC2BF04D0E31EC2BF0BE0E4AECA9
:106570002BF0000E63EC2BF0B9EC48F0000E63EC4E
:106580002BF0B9EC48F0B9EC48F0000E63EC2BF0BE
:10659000B9EC48F0000E63EC2BF0B9EC48F0000EBB
:1065A00063EC2BF0B9EC48F0000E63EC2BF04A5092
:1065B000406E120025EC2BF04D0E31EC2BF0BE0E90
:1065C0004AEC2BF0000E495CD8B407EF33F0010E13
:1065D000495CD8B40CEF33F0020E495CD8B411EF2B
:1065E00033F0030E495CD8B416EF33F0040E495C67
:1065F000D8B41BEF33F0050E495CD8B420EF33F06C
:10660000060E495CD8B425EF33F02AEF33F04BAED9
:106610002FEF33F04FEF33F04BAC2FEF33F04FEF62
:1066200033F04BAA2FEF33F04FEF33F04BA82FEF9F
:1066300033F04FEF33F04BA62FEF33F04FEF33F043
:106640004BA42FEF33F04FEF33F04BA22FEF33F08B
:106650004FEF33F04BA02FEF33F04FEF33F0000E3E
:1066600063EC2BF0B9EC42F0000E63EC2BF0B9ECCC
:1066700048F059EC46F0000E63EC2BF089EC46F044
:10668000000E63EC2BF0B9EC48F0FF0E63EC2BF03E
:1066900049EC43F0FF0E63EC2BF06DEF33F0FF0E8F
:1066A00063EC2BF059EC43F0FF0E63EC2BF0B9ECEC
:1066B00048F059EC46F0000E63EC2BF089EC46F004
:1066C000000E63EC2BF0B9EC48F0000E63EC2BF0FD
:1066D000A9EC42F0000E63EC2BF04A50406E3FA450
:1066E000120080BA85EF33F0070E565CD8B47CEF09
:1066F00033F0562A87EF33F0566A3EBA87EF33F00D
:106700003F944A50406E3E8A12003E9A566A80B8C4
:1067100009EF34F0070E575CD8B492EF33F0572AE4
:106720000BEF34F0576A3EB80BEF34F0000E495CC3
:10673000D8B4BBEF33F0010E495CD8B4C4EF33F0EA
:10674000020E495CD8B4CDEF33F0030E495CD8B4E7
:10675000D6EF33F0040E495CD8B4DFEF33F0050E0A
:10676000495CD8B4E8EF33F0060E495CD8B4F1EFD9
:1067700033F0FAEF33F04BAEC1EF33F04A8E03EF54
:1067800034F04A9E03EF34F04BACCAEF33F04A8C3E
:1067900003EF34F04A9C03EF34F04BAAD3EF33F00D
:1067A0004A8A03EF34F04A9A03EF34F04BA8DCEF47
:1067B00033F04A8803EF34F04A9803EF34F04BA6E5
:1067C000E5EF33F04A8603EF34F04A9603EF34F0F6
:1067D0004BA4EEEF33F04A8403EF34F04A9403EF16
:1067E00034F04BA2F7EF33F04A8203EF34F04A92D1
:1067F00003EF34F04BA000EF34F04A8003EF34F0A5
:106800004A9003EF34F03F944A50406E3E880BEFBD
:1068100034F03E98576A80B058EF34F0070E555C5C
:10682000D8B416EF34F0552A5AEF34F0556A3EB01A
:106830005AEF34F0000E495CD8B43FEF34F0010E4B
:10684000495CD8B442EF34F0020E495CD8B445EF4D
:1068500034F0030E495CD8B448EF34F0040E495CC0
:10686000D8B44BEF34F0050E495CD8B44EEF34F099
:10687000060E495CD8B451EF34F054EF34F04B7E3F
:1068800055EF34F04B7C55EF34F04B7A55EF34F044
:106890004B7855EF34F04B7655EF34F04B7455EFA1
:1068A00034F04B7255EF34F04B703E805AEF34F0B9
:1068B0003E90556A84B6A7EF34F0070E545CD8B406
:1068C00065EF34F0542AAAEF34F0546A3EBCA9EFC5
:1068D00034F0000E495CD8B48EEF34F0010E495C00
:1068E000D8B491EF34F0020E495CD8B494EF34F090
:1068F000030E495CD8B497EF34F0040E495CD8B469
:106900009AEF34F0050E495CD8B49DEF34F0060ED2
:10691000495CD8B4A0EF34F0A3EF34F04B7EA4EF81
:1069200034F04B7CA4EF34F04B7AA4EF34F04B7886
:10693000A4EF34F04B76A4EF34F04B74A4EF34F0B2
:106940004B72A4EF34F04B703E8CA9EF34F03E9CB8
:10695000546A120080B824EF35F0070E575CD8B4A3
:10696000B5EF34F0572A26EF35F0576A3EB826EFD8
:1069700035F0000E465CD8B4ECEF34F0010E465C06
:10698000D8B4F0EF34F0020E465CD8B4F4EF34F033
:10699000030E465CD8B4F8EF34F0040E465CD8B46D
:1069A000FCEF34F0050E465CD8B400EF35F0060E6F
:1069B000465CD8B404EF35F0070E465CD8B408EF57
:1069C00035F0080E465CD8B40CEF35F0090E465C85
:1069D000D8B410EF35F012004A50116E12EF35F0B6
:1069E0004A50126E12EF35F04A50136E12EF35F026
:1069F0004A50146E12EF35F04A50156E12EF35F012
:106A00004A50166E12EF35F04A50176E12EF35F0FD
:106A10004A50186E12EF35F04A50196E12EF35F0E9
:106A20004A501A6E6AEC2CF04A50406E3E88000EB6
:106A3000465CD8B420EF35F0070E496E26EF35F0EE
:106A4000050E496E26EF35F03E98576A120025EC88
:106A50002BF0670E31EC2BF0BC0E4AEC2BF03FBC58
:106A600046EF35F0000E63EC2BF0F9EC46F0000E2B
:106A700063EC2BF0C9EC45F0000E63EC2BF099ECC5
:106A800046F0000E63EC2BF058EF35F0FF0E63EC90
:106A90002BF099EC48F0FF0E63EC2BF059EC47F02B
:106AA000FF0E63EC2BF039EC48F0FF0E63EC2BF09B
:106AB00028EC2BF0440E31EC2BF0BC0E4AEC2BF002
:106AC0003FBC77EF35F0FF0E63EC2BF0E9EC47F0BD
:106AD000FF0E63EC2BF0C9EC48F0FF0E63EC2BF0DB
:106AE000F9EC47F0FF0E63EC2BF089EF35F0000E68
:106AF00063EC2BF049EC46F0000E63EC2BF0B9ECA4
:106B000048F0000E63EC2BF059EC46F0000E63ECFD
:106B10002BF080B0A2EF35F0070E555CD8B494EF9F
:106B200035F0552AA4EF35F0556A3EB0A4EF35F0A4
:106B30003FBC9EEF35F03F8C9FEF35F03F9C3E8091
:106B4000A4EF35F03E90556A84B6BDEF35F0070EE0
:106B5000545CD8B4AFEF35F0542ABFEF35F0546A27
:106B60003EBCBFEF35F03FBCB9EF35F03F8CBAEF1C
:106B700035F03F9C3E8CBFEF35F03E9C546A1200CE
:106B800080B83DEF36F0070E575CD8B4CBEF35F048
:106B9000572A3FEF36F0576A3EB83FEF36F03FAC2A
:106BA00037EF36F04DEC2CF0000E475CD8B40DEF0B
:106BB00036F0010E475CD8B411EF36F0020E475C98
:106BC000D8B415EF36F0030E475CD8B419EF36F0A1
:106BD000040E475CD8B41DEF36F0050E475CD8B400
:106BE00021EF36F0060E475CD8B425EF36F0070EDD
:106BF000475CD8B429EF36F0080E475CD8B42DEFC7
:106C000036F0090E475CD8B431EF36F00A0E475C17
:106C1000D8B435EF36F037EF36F0F1EC48F037EF17
:106C200036F004EC49F037EF36F017EC49F037EF67
:106C300036F02AEC49F037EF36F03DEC49F037EF0B
:106C400036F050EC49F037EF36F063EC49F037EFAF
:106C500036F076EC49F037EF36F089EC49F037EF53
:106C600036F09CEC49F037EF36F0AFEC49F0446A6F
:106C7000476A3F9C3E8823EF01F03E98576A120016
:106C800083A260EF36F03FB812004CB252EF36F0FC
:106C90001550380B406E180E406E1550C70B156E10
:106CA0005AEF36F015503F0B406E1B0E406E1550DC
:106CB000C00B156E405015126AEC2CF03F88120084
:106CC0003F9812001550380B406E404240424042FF
:106CD0004050070B406E1550F80B156E40501512C2
:106CE0001200106E000E105CD8A48FEF36F005B8BD
:106CF00080EF36F005BA84EF36F009EC42F012006E
:106D0000B9EC48F0058C120005BC8BEF36F0059C01
:106D100009EC42F01200059CB9EC48F01200010E9B
:106D2000105CD8A497EF36F019EC42F01200020E76
:106D3000105CD8A49FEF36F029EC42F01200030E4D
:106D4000105CD8A4A7EF36F039EC42F01200040E24
:106D5000105CD8A4AFEF36F049EC42F01200050EFB
:106D6000105CD8A4B7EF36F059EC42F01200060ED2
:106D7000105CD8A4BFEF36F069EC42F01200070EA9
:106D8000105CD8A4C7EF36F079EC42F01200080E80
:106D9000105CD8A4CFEF36F089EC42F0120099ECE9
:106DA00042F01200106E000E105CD8A4DBEF36F03B
:106DB000A9EC42F01200010E105CD8A4E3EF36F00B
:106DC000B9EC42F01200020E105CD8A4EBEF36F0E2
:106DD000C9EC42F01200030E105CD8A4F3EF36F0B9
:106DE000D9EC42F01200040E105CD8A4FBEF36F090
:106DF000E9EC42F01200050E105CD8A403EF37F066
:106E0000F9EC42F01200060E105CD8A40BEF37F03C
:106E100009EC43F01200070E105CD8A413EF37F012
:106E200019EC43F01200080E105CD8A41BEF37F0E9
:106E300029EC43F0120039EC43F01200106E000E02
:106E4000105CD8A427EF37F049EC43F01200010E94
:106E5000105CD8A42FEF37F059EC43F01200020E6B
:106E6000105CD8A437EF37F069EC43F01200030E42
:106E7000105CD8A43FEF37F079EC43F01200040E19
:106E8000105CD8A447EF37F089EC43F01200050EF0
:106E9000105CD8A44FEF37F099EC43F01200060EC7
:106EA000105CD8A457EF37F0A9EC43F01200070E9E
:106EB000105CD8A45FEF37F0B9EC43F01200080E75
:106EC000105CD8A467EF37F0C9EC43F01200D9EC9E
:106ED00043F01200062A0A0E065CD8A46AEF37F0C7
:106EE000066A1200062AFF0E065CD8A472EF37F07D
:106EF000066A072A640E075CD8A472EF37F0066AA8
:106F0000076A1200062AFF0E065CD8A482EF37F04B
:106F1000066A072AFF0E075CD8A482EF37F0066ADC
:106F2000076A120025EC2BF0400E31EC2BF0BF0E5F
:106F30004AEC2BF0B9EC45F0000E63EC2BF089EC39
:106F400045F0000E63EC2BF009EC46F0000E63EC0C
:106F50002BF029EC43F0000E63EC2BF0E9EC42F04F
:106F6000000E63EC2BF0B9EC42F0000E63EC2BF05A
:106F700009EC43F0B9EC48F089EC46F0000E63EC04
:106F80002BF0C9EC45F0000E63EC2BF0C9EC46F099
:106F900028EC2BF0400E31EC2BF0BF0E4AEC2BF01E
:106FA000400E63EC2BF0000E63EC2BF0B9EC42F0DA
:106FB000000E63EC2BF0400E63EC2BF0000E63EC44
:106FC0002BF0A9EC42F0000E63EC2BF0400E036EA8
:106FD0007F0E046E25EC2BF0035031EC2BF0BC0E31
:106FE0004AEC2BF0010E63EC2BF028EC2BF0045054
:106FF00031EC2BF0BC0E4AEC2BF0010E63EC2BF0C5
:10700000032A040672EC37F0800E035CD8A4EAEF82
:1070100037F082EC37F082EC37F082EC37F082EC1C
:1070200037F082EC37F0400E036E7F0E046E25ECD5
:107030002BF0035031EC2BF0BC0E4AEC2BF0000E81
:1070400063EC2BF028EC2BF0045031EC2BF0BC0E51
:107050004AEC2BF0000E63EC2BF0032A040672ECD2
:1070600037F0800E035CD8A417EF38F03F8E82EC27
:1070700037F082EC37F082EC37F082EC37F050805A
:1070800025EC2BF04A0E31EC2BF0BB0E4AEC2BF02A
:1070900039EC44F0000E63EC2BF0100E63EC2BF097
:1070A000100E63EC2BF0100E63EC2BF0100E63EC63
:1070B0002BF0100E63EC2BF0000E63EC2BF0B9EC10
:1070C00044F0000E63EC2BF0B9EC48F0000E63ECDA
:1070D0002BF029EC44F0000E63EC2BF0B9EC44F0FB
:1070E000000E63EC2BF049EC44F0000E63EC2BF047
:1070F00069EC44F0000E63EC2BF0B9EC44F0000EA8
:1071000063EC2BF028EC2BF0400E31EC2BF0BB0E97
:107110004AEC2BF029EC44F0000E63EC2BF029EC48
:1071200044F0000E63EC2BF0F9EC44F0000E63EC3D
:107130002BF069EC44F0000E63EC2BF0B9EC44F05A
:10714000000E63EC2BF049EC44F0000E63EC2BF0E6
:10715000509025EC2BF0560E31EC2BF0BC0E4AEC87
:107160002BF0E9EC43F0000E63EC2BF029EC45F03A
:10717000000E63EC2BF019EC44F0000E63EC2BF0E6
:1071800069EC44F0000E63EC2BF0C9EC44F0000E07
:1071900063EC2BF0B9EC48F0000E63EC2BF099ECAB
:1071A00044F0000E63EC2BF028EC2BF0400E31EC99
:1071B0002BF0BC0E4AEC2BF0E9EC43F0000E63EC34
:1071C0002BF0F9EC43F0000E63EC2BF0C9EC44F02B
:1071D000000E63EC2BF0F9EC44F0000E63EC2BF0A6
:1071E000E9EC43F0000E63EC2BF019EC45F0000ED7
:1071F00063EC2BF0C9EC44F0000E63EC2BF0F9ECDF
:1072000044F0000E63EC2BF069EC45F0000E63ECEB
:107210002BF0512A080E515CD8A437EF38F03F9E6E
:10722000516A82EC37F082EC37F082EC37F082EC76
:1072300037F082EC37F082EC37F082EC37F082ECFA
:1072400037F082EC37F082EC37F082EC37F082ECEA
:1072500037F082EC37F082EC37F082EC37F082ECDA
:1072600037F082EC37F082EC37F082EC37F082ECCA
:1072700037F082EC37F082EC37F082EC37F082ECBA
:1072800037F082EC37F082EC37F082EC37F082ECAA
:1072900037F082EC37F082EC37F082EC37F082EC9A
:1072A00037F082EC37F082EC37F082EC37F082EC8A
:1072B00037F082EC37F082EC37F082EC37F082EC7A
:1072C00037F082EC37F082EC37F082EC37F082EC6A
:1072D00037F082EC37F082EC37F082EC37F082EC5A
:1072E00037F082EC37F082EC37F082EC37F082EC4A
:1072F00037F082EC37F082EC37F082EC37F082EC3A
:1073000037F082EC37F082EC37F082EC37F082EC29
:1073100037F082EC37F082EC37F082EC37F082EC19
:1073200037F082EC37F082EC37F082EC37F082EC09
:1073300037F082EC37F082EC37F082EC37F082ECF9
:1073400037F082EC37F082EC37F04DEC2CF082EC29
:1073500037F082EC37F082EC37F082EC37F0120035
:10736000096E640E095ED8A0B9EF39F00A2AB1EFB0
:1073700039F0640E09260A0E095ED8A0C3EF39F071
:107380000B2ABBEF39F00A0E0926010E095ED8A0C0
:10739000CDEF39F00C2AC5EF39F012000D6E100E4A
:1073A0000D5ED8A0D7EF39F00B2ACFEF39F0100ED1
:1073B0000D26010E0D5ED8A0E1EF39F00C2AD9EFB1
:1073C00039F0120005880A5071EC36F0000E63ECBB
:1073D0002BF00598058A0B5071EC36F0000E63EC2B
:1073E0002BF0059A0C5071EC36F0000E63EC2BF08C
:1073F0000A6A0B6A0C6A12000A50D2EC36F0000ED0
:1074000063EC2BF00B50D2EC36F0000E63EC2BF05B
:107410000C50D2EC36F0000E63EC2BF00A6A0B6ACB
:107420000C6A12000A501EEC37F0FF0E63EC2BF0D2
:107430000B501EEC37F0FF0E63EC2BF00C501EECE3
:1074400037F0FF0E63EC2BF00A6A0B6A0C6A12002D
:10745000406E452A090E455CD8B43EEF3AF040BE76
:1074600036EF3AF0A9EC42F038EF3AF0B9EC42F0DE
:10747000000E63EC2BF0404629EF3AF0456A12000B
:10748000406E080E455CD8B47DEF3AF040BE62EF26
:107490003AF04550495CD8B458EF3AF0000E63EC2E
:1074A0002BF0A9EC42F0000E63EC2BF079EF3AF0F0
:1074B000FF0E63EC2BF049EC43F0FF0E63EC2BF076
:1074C00079EF3AF04550495CD8B471EF3AF0000ECC
:1074D00063EC2BF0B9EC42F0000E63EC2BF079EF8B
:1074E0003AF0FF0E63EC2BF059EC43F0FF0E63EC27
:1074F0002BF0452A404641EF3AF0456A12007D0ED6
:107500004F5CD8B486EF3AF04F2A12003F8A4F6A98
:10751000120028EC2BF0530E31EC2BF0BE0E4AEC8F
:107520002BF0080E495CD8A4E1EF3AF0FF0E63ECB3
:107530002BF039EC48F0FF0E63EC2BF059EC47F0E0
:10754000FF0E63EC2BF049EC48F0FF0E63EC2BF0E0
:1075500025EC2BF0460E31EC2BF0BC0E4AEC2BF058
:10756000000E63EC2BF0B9EC48F0000E63EC2BF04E
:10757000B9EC48F0000E63EC2BF0B9EC48F0000ECB
:1075800063EC2BF0B9EC48F0000E63EC2BF0B9EC97
:1075900048F0000E63EC2BF0B9EC48F0000E63EC01
:1075A0002BF0B9EC48F0000E63EC2BF0B9EC48F08E
:1075B000000E63EC2BF0B9EC48F0000E63EC2BF0FE
:1075C0001200000E63EC2BF099EC46F0000E63EC19
:1075D0002BF0C9EC45F0000E63EC2BF0A9EC46F063
:1075E000000E63EC2BF0120028EC2BF0400E31EC77
:1075F0002BF0BB0E4AEC2BF01200000E63EC2BF0CC
:1076000049EC46F0000E63EC2BF059EC46F0000E0E
:1076100063EC2BF0B9EC48F0000E63EC2BF07FEC40
:107620003CF0B9EC48F0000E63EC2BF0B9EC48F0FC
:10763000B9EC48F0DAEC3CF01200FF0E63EC2BF0F2
:1076400019EC48F0FF0E63EC2BF039EC47F0FF0E1D
:1076500063EC2BF029EC48F0FF0E63EC2BF039ECD7
:1076600047F0FF0E63EC2BF0C9EC48F0FF0E63EC23
:107670002BF099EC3CF0DAEC3CF01200FF0E63ECDE
:107680002BF039EC47F0FF0E63EC2BF039EC47F0B0
:10769000FF0E63EC2BF029EC48F0FF0E63EC2BF0AF
:1076A00039EC47F0FF0E63EC2BF0C9EC48F0FF0E0D
:1076B00063EC2BF099EC3CF0DAEC3CF01200FF0E9E
:1076C00063EC2BF059EC48F0FF0E63EC2BF0E9EC87
:1076D00047F0FF0E63EC2BF0C9EC47F0FF0E63ECB4
:1076E0002BF0F9EC47F0FF0E63EC2BF039EC47F090
:1076F000FF0E63EC2BF0B9EC47F0FF0E63EC2BF0C0
:10770000B9EC48F0000E63EC2BF0B9EC48F0000E39
:1077100063EC2BF0B9EC48F0000E63EC2BF0B9EC05
:1077200048F0000E63EC2BF0DAEC3CF01200FF0E98
:1077300063EC2BF069EC48F0FF0E63EC2BF019ECD6
:1077400047F0FF0E63EC2BF0C9EC47F0FF0E63EC43
:107750002BF099EC47F0FF0E63EC2BF049EC47F06F
:10776000FF0E63EC2BF099EC47F0FF0E63EC2BF06F
:1077700049EC48F0FF0E63EC2BF099EC48F0FF0E5B
:1077800063EC2BF0C9EC48F059EC47F0FF0E63ECCA
:107790002BF0810E63EC2BF0ED0E63EC2BF0ED0E75
:1077A00063EC2BF0ED0E63EC2BF0F4EC3AF0930E5F
:1077B00063EC2BF0FF0E63EC2BF0A3EC3CF0B9EC88
:1077C00048F0000E63EC2BF01200FF0E63EC2BF080
:1077D00029EC47F0FF0E63EC2BF099EC47F0FF0E1D
:1077E00063EC2BF0C9EC48F0FF0E63EC2BF009ECD6
:1077F00048F0FF0E63EC2BF089EC47F0FF0E63ECD2
:107800002BF019EC47F0FF0E63EC2BF039EC48F04D
:10781000FF0E63EC2BF059EC47F0FF0E63EC2BF0FE
:10782000C9EC48F059EC47F0FF0E63EC2BF0810EE9
:1078300063EC2BF0ED0E63EC2BF0ED0E63EC2BF014
:10784000ED0E63EC2BF0F4EC3AF0930E63EC2BF0BE
:10785000FF0E63EC2BF0A3EC3CF0B9EC48F0000E0B
:1078600063EC2BF01200FF0E63EC2BF009EC48F0F8
:10787000FF0E63EC2BF019EC47F0FF0E63EC2BF0DE
:1078800029EC48F0FF0E63EC2BF099EC47F0FF0E6B
:1078900063EC2BF049EC48F0FF0E63EC2BF099EC15
:1078A00048F0FF0E63EC2BF0C9EC48F059EC47F0C0
:1078B000FF0E63EC2BF029EC48F0FF0E63EC2BF08D
:1078C00029EC48F0FF0E63EC2BF0C30E63EC2BF0B9
:1078D000BD0E63EC2BF0BD0E63EC2BF0BD0E63EC24
:1078E0002BF0F4EC3AF0C30E63EC2BF0FF0E63ECDC
:1078F0002BF0ADEC3CF0000E63EC2BF01200C9EC69
:1079000045F0000E63EC2BF089EC46F0000E63ECC2
:107910002BF089EC46F0000E63EC2BF059EC46F0AE
:10792000000E63EC2BF089EC46F0000E63EC2BF0BC
:10793000120059EC47F0FF0E63EC2BF029EC48F0F5
:10794000FF0E63EC2BF029EC48F0FF0E63EC2BF0FC
:10795000F9EC47F0FF0E63EC2BF029EC48F0FF0E3A
:1079600063EC2BF0120099EC3CF0C9EC48F0FF0EF0
:1079700063EC2BF039EC47F0FF0E63EC2BF0F9ECE5
:1079800047F0FF0E63EC2BF049EC47F0FF0E63EC81
:107990002BF059EC47F0FF0E63EC2BF0FF0E63EC7D
:1079A0002BF0FF0E63EC2BF0FF0E63EC2BF0F4ECEE
:1079B0003AF01200F4EC3AF0B9EC48F0000E63EC47
:1079C0002BF0B9EC48F0000E63EC2BF0B9EC48F06A
:1079D000000E63EC2BF0B9EC48F0000E63EC2BF0DA
:1079E000B9EC48F0000E63EC2BF01200A9EC45F066
:1079F000000E63EC2BF059EC46F0000E63EC2BF01C
:107A000049EC46F0000E63EC2BF0A9EC46F0000EBA
:107A100063EC2BF089EC46F0000E63EC2BF059EC94
:107A200046F0000E63EC2BF029EC46F0000E63EC00
:107A30002BF0B9EC48F0A9EC42F0000E63EC2BF00F
:107A4000B9EC48F028EC2BF0400E31EC2BF0B90EDD
:107A50004AEC2BF0FF0E63EC2BF0810E63EC2BF065
:107A6000810E63EC2BF0000E63EC2BF0A9EC42F0DE
:107A7000000E63EC2BF0A9EC42F0000E63EC2BF04F
:107A8000F9EC45F0000E63EC2BF0810E63EC2BF06B
:107A9000810E63EC2BF0FF0E63EC2BF01200A9ECCF
:107AA00045F0000E63EC2BF059EC46F0000E63EC51
:107AB0002BF049EC46F0000E63EC2BF0A9EC46F0FD
:107AC000000E63EC2BF089EC46F0000E63EC2BF01B
:107AD00059EC46F0000E63EC2BF029EC46F0000E5A
:107AE00063EC2BF0B9EC48F0B9EC42F0000E63EC1B
:107AF0002BF0B9EC48F028EC2BF0400E31EC2BF0D9
:107B0000B90E4AEC2BF0FF0E63EC2BF0810E63EC08
:107B10002BF0810E63EC2BF0000E63EC2BF0A9EC44
:107B200042F0000E63EC2BF0B9EC42F0000E63EC77
:107B30002BF0F9EC45F0000E63EC2BF0810E63ECBA
:107B40002BF0810E63EC2BF0FF0E63EC2BF0120098
:107B5000A9EC45F0000E63EC2BF059EC46F0000E5A
:107B600063EC2BF049EC46F0000E63EC2BF0A9EC33
:107B700046F0000E63EC2BF089EC46F0000E63EC4F
:107B80002BF059EC46F0000E63EC2BF029EC46F09C
:107B9000000E63EC2BF0B9EC48F0C9EC42F0000E9B
:107BA00063EC2BF0B9EC48F028EC2BF0400E31ECF4
:107BB0002BF0B90E4AEC2BF0FF0E63EC2BF0810E8C
:107BC00063EC2BF0810E63EC2BF0000E63EC2BF0DA
:107BD000A9EC42F0000E63EC2BF0C9EC42F0000E71
:107BE00063EC2BF0F9EC45F0000E63EC2BF0810E0A
:107BF00063EC2BF0810E63EC2BF0FF0E63EC2BF0AB
:107C00001200A9EC45F0000E63EC2BF059EC46F0A5
:107C1000000E63EC2BF049EC46F0000E63EC2BF009
:107C2000A9EC46F0000E63EC2BF089EC46F0000E58
:107C300063EC2BF059EC46F0000E63EC2BF029ECD2
:107C400046F0000E63EC2BF0B9EC48F0D9EC42F0B2
:107C5000000E63EC2BF0B9EC48F028EC2BF0400E52
:107C600031EC2BF0B90E4AEC2BF0FF0E63EC2BF04D
:107C7000810E63EC2BF0810E63EC2BF0000E63ECB5
:107C80002BF0A9EC42F0000E63EC2BF0D9EC42F0A3
:107C9000000E63EC2BF0F9EC45F0000E63EC2BF0DA
:107CA000810E63EC2BF0810E63EC2BF0FF0E63EC86
:107CB0002BF01200A9EC45F0000E63EC2BF059EC10
:107CC00046F0000E63EC2BF049EC46F0000E63EC3E
:107CD0002BF0A9EC46F0000E63EC2BF089EC46F09B
:107CE000000E63EC2BF059EC46F0000E63EC2BF029
:107CF00029EC46F0000E63EC2BF0B9EC48F0E9EC0F
:107D000042F0000E63EC2BF0B9EC48F028EC2BF0BD
:107D1000400E31EC2BF0B90E4AEC2BF0FF0E63EC69
:107D20002BF0810E63EC2BF0810E63EC2BF0000E38
:107D300063EC2BF0A9EC42F0000E63EC2BF0E9ECC5
:107D400042F0000E63EC2BF0F9EC45F0000E63EC12
:107D50002BF0810E63EC2BF0810E63EC2BF0FF0E09
:107D600063EC2BF0120099EC46F0000E63EC2BF064
:107D7000C9EC45F0000E63EC2BF089EC46F0000EE8
:107D800063EC2BF009EC46F0000E63EC2BF089EC71
:107D900045F0000E63EC2BF029EC46F0000E63EC8E
:107DA0002BF0B9EC48F089EC45F0000E63EC2BF0B9
:107DB000B9EC46F0000E63EC2BF0B9EC45F028EC82
:107DC0002BF0400E31EC2BF0B90E4AEC2BF0000EEC
:107DD00063EC2BF009EC46F0000E63EC2BF059EC51
:107DE00046F0000E63EC2BF025EC2BF04C0E31EC42
:107DF0002BF0BA0E4AEC2BF0B9EC45F0000E63EC18
:107E00002BF089EC45F0000E63EC2BF0A9EC46F06A
:107E1000000E63EC2BF089EC45F0000E63EC2BF0C8
:107E2000B9EC48F0D9EC45F0000E63EC2BF059ECBE
:107E300046F0000E63EC2BF089EC46F0000E63EC8C
:107E40002BF039EC46F028EC2BF0400E31EC2BF007
:107E5000BA0E4AEC2BF0000E63EC2BF089EC45F0E7
:107E6000000E63EC2BF0A9EC46F0B9EC48F0FF0EE5
:107E700063EC2BF0810E63EC2BF0810E63EC2BF0A6
:107E8000000E63EC2BF0A9EC42F0000E63EC2BF03B
:107E9000F9EC42F0000E63EC2BF0F9EC45F0000E2B
:107EA00063EC2BF0810E63EC2BF0810E63EC2BF076
:107EB000FF0E63EC2BF0120089EC46F0000E63EC31
:107EC0002BF0C9EC45F0000E63EC2BF0A9EC45F06B
:107ED000000E63EC2BF0C9EC45F0000E63EC2BF0C8
:107EE00009EC46F0000E63EC2BF0C9EC46F0000EF6
:107EF00063EC2BF0C9EC45F0000E63EC2BF089EC41
:107F000046F0000E63EC2BF0B9EC48F0C9EC45F0FC
:107F100028EC2BF0400E31EC2BF0B90E4AEC2BF094
:107F2000000E63EC2BF089EC46F0000E63EC2BF0B6
:107F300089EC46F0000E63EC2BF059EC46F0000E95
:107F400063EC2BF089EC46F0000E63EC2BF0B9ECFF
:107F500048F039EC46F0000E63EC2BF089EC45F06C
:107F6000000E63EC2BF099EC46F0000E63EC2BF066
:107F700019EC46F0000E63EC2BF028EC2BF0640EAD
:107F800031EC2BF0BA0E4AEC2BF0FF0E63EC2BF029
:107F9000810E63EC2BF0810E63EC2BF0000E63EC92
:107FA0002BF0A9EC42F0000E63EC2BF009EC43F04F
:107FB000000E63EC2BF0F9EC45F0000E63EC2BF0B7
:107FC000810E63EC2BF0810E63EC2BF0FF0E63EC63
:107FD0002BF0120009EC46F0000E63EC2BF049EC9C
:107FE00046F0000E63EC2BF0A9EC46F0000E63ECBB
:107FF0002BF0C9EC45F0000E63EC2BF089EC46F059
:10800000000E63EC2BF089EC46F0000E63EC2BF0D5
:10801000B9EC46F0000E63EC2BF069EC46F0000E74
:1080200063EC2BF0A9EC46F0B9EC48F028EC2BF00F
:10803000400E31EC2BF0B90E4AEC2BF0000E63EC45
:108040002BF039EC46F0000E63EC2BF089EC45F098
:10805000000E63EC2BF099EC46F0000E63EC2BF075
:1080600019EC46F0B9EC48F0FF0E63EC2BF0810EF2
:1080700063EC2BF0810E63EC2BF0000E63EC2BF025
:10808000A9EC42F0000E63EC2BF019EC43F0000E6B
:1080900063EC2BF0F9EC45F0000E63EC2BF0810E55
:1080A00063EC2BF0810E63EC2BF0FF0E63EC2BF0F6
:1080B000120009EC46F0000E63EC2BF049EC46F0A0
:1080C000000E63EC2BF0A9EC46F0000E63EC2BF0F5
:1080D000C9EC45F0000E63EC2BF089EC46F0000E85
:1080E00063EC2BF089EC46F0000E63EC2BF0B9EC5E
:1080F00046F0000E63EC2BF069EC46F0000E63ECEA
:108100002BF0A9EC46F0B9EC48F028EC2BF0400E2F
:1081100031EC2BF0B90E4AEC2BF0000E63EC2BF097
:1081200039EC46F0000E63EC2BF059EC46F0000EF3
:1081300063EC2BF0B9EC45F0000E63EC2BF0C9ECCE
:1081400045F0000E63EC2BF0B9EC48F039EC46F04A
:10815000000E63EC2BF099EC46F0000E63EC2BF074
:1081600099EC45F0000E63EC2BF028EC2BF0640E3C
:1081700031EC2BF0BA0E4AEC2BF0FF0E63EC2BF037
:10818000810E63EC2BF0810E63EC2BF0000E63ECA0
:108190002BF0A9EC42F0000E63EC2BF029EC43F03D
:1081A000000E63EC2BF0F9EC45F0000E63EC2BF0C5
:1081B000810E63EC2BF0810E63EC2BF0FF0E63EC71
:1081C0002BF0120009EC46F0000E63EC2BF049ECAA
:1081D00046F0000E63EC2BF0A9EC46F0000E63ECC9
:1081E0002BF0C9EC45F0000E63EC2BF089EC46F067
:1081F000000E63EC2BF089EC46F0000E63EC2BF0E4
:10820000B9EC46F0000E63EC2BF069EC46F0000E82
:1082100063EC2BF0A9EC46F0B9EC48F028EC2BF01D
:10822000400E31EC2BF0B90E4AEC2BF0000E63EC53
:108230002BF039EC46F0000E63EC2BF059EC46F0D5
:10824000000E63EC2BF0B9EC45F0000E63EC2BF064
:10825000C9EC45F0000E63EC2BF0B9EC48F029ECCA
:1082600046F0000E63EC2BF099EC46F0000E63EC48
:108270002BF099EC45F0000E63EC2BF028EC2BF082
:10828000640E31EC2BF0BA0E4AEC2BF0FF0E63ECCF
:108290002BF0810E63EC2BF0810E63EC2BF0000EC3
:1082A00063EC2BF0A9EC42F0000E63EC2BF039EC00
:1082B00043F0000E63EC2BF0F9EC45F0000E63EC9C
:1082C0002BF0810E63EC2BF0810E63EC2BF0FF0E94
:1082D00063EC2BF01200FF0E63EC2BF009EC48F07E
:1082E000FF0E63EC2BF039EC47F0FF0E63EC2BF044
:1082F00039EC47F0FF0E63EC2BF089EC47F0FF0EF2
:1083000063EC2BF01200FF0E63EC2BF0F9EC47F05E
:10831000FF0E63EC2BF039EC48F0FF0E63EC2BF012
:10832000C9EC47F0FF0E63EC2BF099EC47F0FF0E21
:1083300063EC2BF009EC48F0FF0E63EC2BF012001D
:10834000FF0E63EC2BF049EC47F0FF0E63EC2BF0D3
:1083500059EC47F0FF0E63EC2BF049EC48F0FF0EB0
:1083600063EC2BF039EC47F0FF0E63EC2BF01200BE
:10837000FF0E63EC2BF039EC47F0FF0E63EC2BF0B3
:1083800039EC47F0FF0E63EC2BF089EC47F0FF0E61
:1083900063EC2BF01200FF0E63EC2BF029EC48F09D
:1083A000FF0E63EC2BF059EC47F0FF0E63EC2BF063
:1083B00029EC48F0FF0E63EC2BF029EC48F0FF0E9F
:1083C00063EC2BF01200FF0E63EC2BF019EC48F07D
:1083D000FF0E63EC2BF039EC47F0FF0E63EC2BF053
:1083E00089EC47F0FF0E63EC2BF01200FF0E63ECFC
:1083F0002BF069EC47F0FF0E63EC2BF039EC47F003
:10840000FF0E63EC2BF089EC47F0FF0E63EC2BF0D2
:1084100012007C0E63EC2BF0820E63EC2BF0820ECC
:1084200063EC2BF0820E63EC2BF07C0E63EC2BF0F4
:108430001200000E63EC2BF0840E63EC2BF0FE0EAA
:1084400063EC2BF0800E63EC2BF0000E63EC2BF052
:108450001200E20E63EC2BF0920E63EC2BF0920E06
:1084600063EC2BF0920E63EC2BF08C0E63EC2BF094
:108470001200440E63EC2BF0820E63EC2BF0920E94
:1084800063EC2BF0920E63EC2BF06C0E63EC2BF094
:108490001200300E63EC2BF0280E63EC2BF0240E50
:1084A00063EC2BF0FE0E63EC2BF0200E63EC2BF054
:1084B00012004E0E63EC2BF08A0E63EC2BF08A0E4A
:1084C00063EC2BF08A0E63EC2BF0720E63EC2BF056
:1084D00012007C0E63EC2BF0920E63EC2BF0920EEC
:1084E00063EC2BF0920E63EC2BF0640E63EC2BF03C
:1084F0001200060E63EC2BF0020E63EC2BF0C20EA2
:1085000063EC2BF0320E63EC2BF00E0E63EC2BF0D1
:1085100012006C0E63EC2BF0920E63EC2BF0920EBB
:1085200063EC2BF0920E63EC2BF06C0E63EC2BF0F3
:1085300012004C0E63EC2BF0920E63EC2BF0920EBB
:1085400063EC2BF0920E63EC2BF07C0E63EC2BF0C3
:1085500012003C0E63EC2BF0420E63EC2BF0420E4B
:1085600063EC2BF0420E63EC2BF03C0E63EC2BF033
:108570001200000E63EC2BF0440E63EC2BF07E0E29
:1085800063EC2BF0400E63EC2BF0000E63EC2BF051
:108590001200720E63EC2BF04A0E63EC2BF04A0EC5
:1085A00063EC2BF04A0E63EC2BF0440E63EC2BF0E3
:1085B0001200220E63EC2BF04A0E63EC2BF04A0EF5
:1085C00063EC2BF04A0E63EC2BF0340E63EC2BF0D3
:1085D0001200300E63EC2BF0280E63EC2BF0240E0F
:1085E00063EC2BF07E0E63EC2BF0200E63EC2BF093
:1085F00012002E0E63EC2BF04A0E63EC2BF04A0EA9
:1086000063EC2BF04A0E63EC2BF0320E63EC2BF094
:1086100012003C0E63EC2BF04A0E63EC2BF04A0E7A
:1086200063EC2BF04A0E63EC2BF0300E63EC2BF076
:108630001200060E63EC2BF0020E63EC2BF0620EC0
:1086400063EC2BF0120E63EC2BF00E0E63EC2BF0B0
:108650001200340E63EC2BF04A0E63EC2BF04A0E42
:1086600063EC2BF04A0E63EC2BF0340E63EC2BF032
:1086700012000C0E63EC2BF0520E63EC2BF0520E3A
:1086800063EC2BF0520E63EC2BF03C0E63EC2BF002
:108690001200C30E63EC2BF0BD0E63EC2BF0BD0E8D
:1086A00063EC2BF0BD0E63EC2BF0C30E63EC2BF0F0
:1086B0001200FF0E63EC2BF0BB0E63EC2BF0810E6F
:1086C00063EC2BF0BF0E63EC2BF0FF0E63EC2BF092
:1086D00012008D0E63EC2BF0B50E63EC2BF0B50E93
:1086E00063EC2BF0B50E63EC2BF0BB0E63EC2BF0C0
:1086F0001200DD0E63EC2BF0B50E63EC2BF0B50E23
:1087000063EC2BF0B50E63EC2BF0CB0E63EC2BF08F
:108710001200CF0E63EC2BF0D70E63EC2BF0DB0EC8
:1087200063EC2BF0810E63EC2BF0DF0E63EC2BF08F
:108730001200D10E63EC2BF0B50E63EC2BF0B50EEE
:1087400063EC2BF0B50E63EC2BF0CD0E63EC2BF04D
:108750001200C30E63EC2BF0B50E63EC2BF0B50EDC
:1087600063EC2BF0B50E63EC2BF0CF0E63EC2BF02B
:108770001200F90E63EC2BF0FD0E63EC2BF09D0E56
:1087800063EC2BF0ED0E63EC2BF0F10E63EC2BF0B1
:108790001200CB0E63EC2BF0B50E63EC2BF0B50E94
:1087A00063EC2BF0B50E63EC2BF0CB0E63EC2BF0EF
:1087B0001200F30E63EC2BF0AD0E63EC2BF0AD0E5C
:1087C00063EC2BF0AD0E63EC2BF0C30E63EC2BF0DF
:1087D0001200F80E63EC2BF0240E63EC2BF0220E4B
:1087E00063EC2BF0240E63EC2BF0F80E63EC2BF013
:1087F0001200FE0E63EC2BF0920E63EC2BF0920E47
:1088000063EC2BF0920E63EC2BF06C0E63EC2BF010
:1088100012007C0E63EC2BF0820E63EC2BF0820EC8
:1088200063EC2BF0820E63EC2BF0440E63EC2BF028
:108830001200FE0E63EC2BF0820E63EC2BF0820E26
:1088400063EC2BF0820E63EC2BF07C0E63EC2BF0D0
:108850001200FE0E63EC2BF0920E63EC2BF0920EE6
:1088600063EC2BF0920E63EC2BF0820E63EC2BF09A
:108870001200FE0E63EC2BF0120E63EC2BF0120EC6
:1088800063EC2BF0120E63EC2BF0020E63EC2BF07A
:1088900012007C0E63EC2BF0820E63EC2BF0820E48
:1088A00063EC2BF0920E63EC2BF0740E63EC2BF068
:1088B0001200FE0E63EC2BF0100E63EC2BF0100E8A
:1088C00063EC2BF0100E63EC2BF0FE0E63EC2BF040
:1088D0001200000E63EC2BF0820E63EC2BF0FE0E08
:1088E00063EC2BF0820E63EC2BF0000E63EC2BF0AC
:1088F0001200600E63EC2BF0800E63EC2BF0800E08
:1089000063EC2BF0800E63EC2BF07E0E63EC2BF00F
:108910001200FE0E63EC2BF0100E63EC2BF0280E11
:1089200063EC2BF0440E63EC2BF0820E63EC2BF027
:108930001200FE0E63EC2BF0800E63EC2BF0800E29
:1089400063EC2BF0800E63EC2BF0800E63EC2BF0CD
:108950001200FE0E63EC2BF0040E63EC2BF0080EFD
:1089600063EC2BF0040E63EC2BF0FE0E63EC2BF0AB
:108970001200FE0E63EC2BF0080E63EC2BF0100ED1
:1089800063EC2BF0200E63EC2BF0FE0E63EC2BF06F
:1089900012007C0E63EC2BF0820E63EC2BF0820E47
:1089A00063EC2BF0820E63EC2BF07C0E63EC2BF06F
:1089B0001200FE0E63EC2BF0120E63EC2BF0120E85
:1089C00063EC2BF0120E63EC2BF00C0E63EC2BF02F
:1089D00012007C0E63EC2BF0820E63EC2BF0A20EE7
:1089E00063EC2BF0420E63EC2BF0BC0E63EC2BF02F
:1089F0001200FE0E63EC2BF0120E63EC2BF0120E45
:108A000063EC2BF0120E63EC2BF0EC0E63EC2BF00E
:108A100012004C0E63EC2BF0920E63EC2BF0920ED6
:108A200063EC2BF0920E63EC2BF0640E63EC2BF0F6
:108A30001200020E63EC2BF0020E63EC2BF0FE0E24
:108A400063EC2BF0020E63EC2BF0020E63EC2BF0C8
:108A500012007E0E63EC2BF0800E63EC2BF0800E88
:108A600063EC2BF0800E63EC2BF07E0E63EC2BF0AE
:108A700012000E0E63EC2BF0300E63EC2BF0C00EE8
:108A800063EC2BF0300E63EC2BF00E0E63EC2BF04E
:108A900012001E0E63EC2BF0E00E63EC2BF0180EB0
:108AA00063EC2BF0E00E63EC2BF01E0E63EC2BF06E
:108AB0001200C60E63EC2BF0280E63EC2BF0100EA8
:108AC00063EC2BF0280E63EC2BF0C60E63EC2BF05E
:108AD00012000E0E63EC2BF0100E63EC2BF0E00E88
:108AE00063EC2BF0100E63EC2BF00E0E63EC2BF00E
:108AF0001200C20E63EC2BF0A20E63EC2BF0920E70
:108B000063EC2BF08A0E63EC2BF0860E63EC2BF0FB
:108B10001200780E63EC2BF0140E63EC2BF0120EA7
:108B200063EC2BF0140E63EC2BF0780E63EC2BF05F
:108B300012007E0E63EC2BF04A0E63EC2BF04A0E13
:108B400063EC2BF04A0E63EC2BF0340E63EC2BF04D
:108B500012003C0E63EC2BF0420E63EC2BF0420E45
:108B600063EC2BF0420E63EC2BF0240E63EC2BF045
:108B700012007E0E63EC2BF0420E63EC2BF0420EE3
:108B800063EC2BF0420E63EC2BF03C0E63EC2BF00D
:108B900012007E0E63EC2BF04A0E63EC2BF04A0EB3
:108BA00063EC2BF04A0E63EC2BF0420E63EC2BF0DF
:108BB00012007E0E63EC2BF00A0E63EC2BF00A0E13
:108BC00063EC2BF00A0E63EC2BF0020E63EC2BF03F
:108BD00012003C0E63EC2BF0420E63EC2BF0420EC5
:108BE00063EC2BF0520E63EC2BF0340E63EC2BF0A5
:108BF00012007E0E63EC2BF0080E63EC2BF0080ED7
:108C000063EC2BF0080E63EC2BF07E0E63EC2BF084
:108C10001200000E63EC2BF0420E63EC2BF07E0E84
:108C200063EC2BF0420E63EC2BF0000E63EC2BF0A8
:108C300012007E0E63EC2BF0100E63EC2BF0080E8E
:108C400063EC2BF0140E63EC2BF0620E63EC2BF054
:108C500012007E0E63EC2BF0400E63EC2BF0400E06
:108C600063EC2BF0400E63EC2BF0400E63EC2BF02A
:108C700012007E0E63EC2BF0040E63EC2BF0080E5A
:108C800063EC2BF0040E63EC2BF07E0E63EC2BF008
:108C900012007E0E63EC2BF0040E63EC2BF0180E2A
:108CA00063EC2BF0200E63EC2BF07E0E63EC2BF0CC
:108CB00012003C0E63EC2BF0420E63EC2BF0420EE4
:108CC00063EC2BF0420E63EC2BF03C0E63EC2BF0CC
:108CD00012007E0E63EC2BF0120E63EC2BF0120EE2
:108CE00063EC2BF0120E63EC2BF00C0E63EC2BF00C
:108CF00012003C0E63EC2BF0420E63EC2BF0520E94
:108D000063EC2BF0220E63EC2BF05C0E63EC2BF08B
:108D100012007E0E63EC2BF0120E63EC2BF0120EA1
:108D200063EC2BF0120E63EC2BF06C0E63EC2BF06B
:108D30001200440E63EC2BF04A0E63EC2BF04A0E4B
:108D400063EC2BF04A0E63EC2BF0320E63EC2BF04D
:108D50001200020E63EC2BF0020E63EC2BF07E0E81
:108D600063EC2BF0020E63EC2BF0020E63EC2BF0A5
:108D700012003E0E63EC2BF0400E63EC2BF0400E25
:108D800063EC2BF0400E63EC2BF03E0E63EC2BF00B
:108D90001200060E63EC2BF0180E63EC2BF0600E45
:108DA00063EC2BF0180E63EC2BF0060E63EC2BF04B
:108DB00012007E0E63EC2BF0200E63EC2BF0100EF5
:108DC00063EC2BF0200E63EC2BF07E0E63EC2BF0AB
:108DD0001200460E63EC2BF0280E63EC2BF0100E05
:108DE00063EC2BF0280E63EC2BF0460E63EC2BF0BB
:108DF0001200060E63EC2BF0080E63EC2BF0700EE5
:108E000063EC2BF0080E63EC2BF0060E63EC2BF0FA
:108E10001200440E63EC2BF0640E63EC2BF0540E46
:108E200063EC2BF04C0E63EC2BF0440E63EC2BF058
:108E30001200870E63EC2BF0EB0E63EC2BF0ED0EC3
:108E400063EC2BF0EB0E63EC2BF0870E63EC2BF056
:108E50001200810E63EC2BF0B50E63EC2BF0B50E17
:108E600063EC2BF0B50E63EC2BF0CB0E63EC2BF028
:108E70001200C30E63EC2BF0BD0E63EC2BF0BD0EA5
:108E800063EC2BF0BD0E63EC2BF0DB0E63EC2BF0F0
:108E90001200810E63EC2BF0BD0E63EC2BF0BD0EC7
:108EA00063EC2BF0BD0E63EC2BF0C30E63EC2BF0E8
:108EB0001200810E63EC2BF0B50E63EC2BF0B50EB7
:108EC00063EC2BF0B50E63EC2BF0BD0E63EC2BF0D6
:108ED0001200810E63EC2BF0F50E63EC2BF0F50E17
:108EE00063EC2BF0F50E63EC2BF0FD0E63EC2BF036
:108EF0001200C30E63EC2BF0BD0E63EC2BF0BD0E25
:108F000063EC2BF0AD0E63EC2BF0CB0E63EC2BF08F
:108F10001200810E63EC2BF0F70E63EC2BF0F70ED2
:108F200063EC2BF0F70E63EC2BF0810E63EC2BF06F
:108F30001200FF0E63EC2BF0BD0E63EC2BF0810EE4
:108F400063EC2BF0BD0E63EC2BF0FF0E63EC2BF00B
:108F50001200CF0E63EC2BF0BF0E63EC2BF0BF0EB4
:108F600063EC2BF0BF0E63EC2BF0C10E63EC2BF027
:108F70001200810E63EC2BF0EF0E63EC2BF0F70E7A
:108F800063EC2BF0EB0E63EC2BF09D0E63EC2BF0FF
:108F90001200810E63EC2BF0BF0E63EC2BF0BF0EC2
:108FA00063EC2BF0BF0E63EC2BF0BF0E63EC2BF0E9
:108FB0001200810E63EC2BF0FB0E63EC2BF0F70E2E
:108FC00063EC2BF0FB0E63EC2BF0810E63EC2BF0CB
:108FD0001200810E63EC2BF0FB0E63EC2BF0E70E1E
:108FE00063EC2BF0DF0E63EC2BF0810E63EC2BF0C7
:108FF0001200C30E63EC2BF0BD0E63EC2BF0BD0E24
:1090000063EC2BF0BD0E63EC2BF0C30E63EC2BF086
:109010001200810E63EC2BF0ED0E63EC2BF0ED0EE5
:1090200063EC2BF0ED0E63EC2BF0F30E63EC2BF006
:109030001200C30E63EC2BF0BD0E63EC2BF0AD0EF3
:1090400063EC2BF0DD0E63EC2BF0A30E63EC2BF046
:109050001200810E63EC2BF0ED0E63EC2BF0ED0EA5
:1090600063EC2BF0ED0E63EC2BF0930E63EC2BF026
:109070001200BB0E63EC2BF0B50E63EC2BF0B50EBB
:1090800063EC2BF0B50E63EC2BF0CD0E63EC2BF004
:109090001200FD0E63EC2BF0FD0E63EC2BF0810E45
:1090A00063EC2BF0FD0E63EC2BF0FD0E63EC2BF06C
:1090B0001200C10E63EC2BF0BF0E63EC2BF0BF0E61
:1090C00063EC2BF0BF0E63EC2BF0C10E63EC2BF0C6
:1090D0001200F90E63EC2BF0E70E63EC2BF09F0E01
:1090E00063EC2BF0E70E63EC2BF0F90E63EC2BF046
:1090F0001200810E63EC2BF0DF0E63EC2BF0EF0E11
:1091000063EC2BF0DF0E63EC2BF0810E63EC2BF0A5
:109110001200B90E63EC2BF0D70E63EC2BF0EF0EC0
:1091200063EC2BF0D70E63EC2BF0B90E63EC2BF055
:109130001200F90E63EC2BF0F70E63EC2BF08F0EA0
:1091400063EC2BF0F70E63EC2BF0F90E63EC2BF0D5
:109150001200000E63EC2BF0000E63EC2BF0040EFB
:1091600063EC2BF00A0E63EC2BF0040E63EC2BF097
:109170001200000E63EC2BF0000E63EC2BF0000EDF
:1091800063EC2BF0000E63EC2BF0000E63EC2BF085
:109190001200FF0E63EC2BF0FF0E63EC2BF0FF0EC2
:1091A00063EC2BF0FF0E63EC2BF0FF0E63EC2BF067
:1091B0001200280E63EC2BF01200FE0E63EC2BF075
:1091C000FE0E63EC2BF0000E63EC2BF01200000E91
:1091D00063EC2BF0000E63EC2BF0000E63EC2BF035
:1091E0001200000EAA6E000EA96E1150A86EA69E67
:1091F000A69CA684550EA76EAA0EA76EA682A6B23E
:10920000FFEF48F0A6941200000EAA6E010EA96EA0
:109210001250A86EA69EA69CA684550EA76EAA0EF6
:10922000A76EA682A6B212EF49F0A6941200000E15
:10923000AA6E020EA96E1350A86EA69EA69CA684C6
:10924000550EA76EAA0EA76EA682A6B225EF49F00C
:10925000A6941200000EAA6E030EA96E1450A86EFA
:10926000A69EA69CA684550EA76EAA0EA76EA682E1
:10927000A6B238EF49F0A6941200000EAA6E040EB2
:10928000A96E1550A86EA69EA69CA684550EA76E24
:10929000AA0EA76EA682A6B24BEF49F0A6941200C2
:1092A000000EAA6E050EA96E1650A86EA69EA69C6C
:1092B000A684550EA76EAA0EA76EA682A6B25EEF72
:1092C00049F0A6941200000EAA6E060EA96E175061
:1092D000A86EA69EA69CA684550EA76EAA0EA76E83
:1092E000A682A6B271EF49F0A6941200000EAA6EF3
:1092F000070EA96E1850A86EA69EA69CA684550EB1
:10930000A76EAA0EA76EA682A6B284EF49F0A69415
:109310001200000EAA6E080EA96E1950A86EA69E25
:10932000A69CA684550EA76EAA0EA76EA682A6B20C
:1093300097EF49F0A6941200000EAA6E090EA96ECE
:109340001A50A86EA69EA69CA684550EA76EAA0EBD
:10935000A76EA682A6B2AAEF49F0A6941200000E4C
:10936000AA6E0A0EA96E4C9E4C50A86EA69EA69C94
:10937000A684550EA76EAA0EA76EA682A6B2BEEF51
:0693800049F0A694120062
:020000040030CA
:03000100331800B1
:02000500358044
:060008000FC00FE00F40E5
:0200000400F00A
:0C00000008044BBB9B887F7F00000000C1
:00000001FF
